:0100000000FF
:0100010000FE
:0100020000FD
:0100030000FC
:0100040000FB
:0100050000FA
:0100060000F9
:0100070000F8
:0100080000F7
:0100090000F6
:01000A0000F5
:01000B0000F4
:01000C0000F3
:01000D0000F2
:01000E0000F1
:01000F0000F0
:0100100000EF
:0100110000EE
:0100120000ED
:0100130000EC
:0100140000EB
:0100150000EA
:0100160000E9
:0100170000E8
:0100180000E7
:0100190000E6
:01001A0000E5
:01001B0000E4
:01001C0000E3
:01001D0000E2
:01001E0000E1
:01001F0000E0
:0100200000DF
:0100210000DE
:0100220000DD
:0100230000DC
:0100240000DB
:0100250000DA
:0100260000D9
:0100270000D8
:0100280000D7
:0100290000D6
:01002A0000D5
:01002B0000D4
:01002C0000D3
:01002D0000D2
:01002E0000D1
:01002F0000D0
:0100300000CF
:0100310000CE
:0100320000CD
:0100330000CC
:0100340000CB
:0100350000CA
:0100360000C9
:0100370000C8
:0100380000C7
:0100390000C6
:01003A0000C5
:01003B0000C4
:01003C0000C3
:01003D0000C2
:01003E0000C1
:01003F0000C0
:0100400000BF
:0100410000BE
:0100420000BD
:0100430000BC
:0100440000BB
:0100450000BA
:0100460000B9
:0100470000B8
:0100480000B7
:0100490000B6
:01004A0000B5
:01004B0000B4
:01004C0000B3
:01004D0000B2
:01004E0000B1
:01004F0000B0
:0100500000AF
:0100510000AE
:0100520000AD
:0100530000AC
:0100540000AB
:0100550000AA
:0100560000A9
:0100570000A8
:0100580000A7
:0100590000A6
:01005A0000A5
:01005B0000A4
:01005C0000A3
:01005D0000A2
:01005E0000A1
:01005F0000A0
:01006000009F
:01006100009E
:01006200009D
:01006300009C
:01006400009B
:01006500009A
:010066000099
:010067000098
:010068000097
:010069000096
:01006A000095
:01006B000094
:01006C000093
:01006D000092
:01006E000091
:01006F000090
:01007000008F
:01007100008E
:01007200008D
:01007300008C
:01007400008B
:01007500008A
:010076000089
:010077000088
:010078000087
:010079000086
:01007A000085
:01007B000084
:01007C000083
:01007D000082
:01007E000081
:01007F000080
:01008000007F
:01008100007E
:01008200007D
:01008300007C
:01008400007B
:01008500007A
:010086000079
:010087000078
:010088000077
:010089000076
:01008A000075
:01008B000074
:01008C000073
:01008D000072
:01008E000071
:01008F000070
:01009000006F
:01009100006E
:01009200006D
:01009300006C
:01009400006B
:01009500006A
:010096000069
:010097000068
:010098000067
:010099000066
:01009A000065
:01009B000064
:01009C000063
:01009D000062
:01009E000061
:01009F000060
:0100A000005F
:0100A100005E
:0100A200005D
:0100A300005C
:0100A400005B
:0100A500005A
:0100A6000059
:0100A7000058
:0100A8000057
:0100A9000056
:0100AA000055
:0100AB000054
:0100AC000053
:0100AD000052
:0100AE000051
:0100AF000050
:0100B000004F
:0100B100004E
:0100B200004D
:0100B300004C
:0100B400004B
:0100B500004A
:0100B6000049
:0100B7000048
:0100B8000047
:0100B9000046
:0100BA000045
:0100BB000044
:0100BC000043
:0100BD000042
:0100BE000041
:0100BF000040
:0100C000003F
:0100C100003E
:0100C200003D
:0100C300003C
:0100C400003B
:0100C500003A
:0100C6000039
:0100C7000038
:0100C8000037
:0100C9000036
:0100CA000035
:0100CB000034
:0100CC000033
:0100CD000032
:0100CE000031
:0100CF000030
:0100D000002F
:0100D100002E
:0100D200002D
:0100D300002C
:0100D400002B
:0100D500002A
:0100D6000029
:0100D7000028
:0100D8000027
:0100D9000026
:0100DA000025
:0100DB000024
:0100DC000023
:0100DD000022
:0100DE000021
:0100DF000020
:0100E000001F
:0100E100001E
:0100E200001D
:0100E300001C
:0100E400001B
:0100E500001A
:0100E6000019
:0100E7000018
:0100E8000017
:0100E9000016
:0100EA000015
:0100EB000014
:0100EC000013
:0100ED000012
:0100EE000011
:0100EF000010
:0100F000000F
:0100F100000E
:0100F200000D
:0100F300000C
:0100F400000B
:0100F500000A
:0100F6000009
:0100F7000008
:0100F8000007
:0100F9000006
:0100FA000005
:0100FB000004
:0100FC000003
:0100FD000002
:0100FE000001
:0100FF000000
:0101000000FE
:0101010000FD
:0101020000FC
:0101030000FB
:0101040000FA
:0101050000F9
:0101060000F8
:0101070000F7
:0101080000F6
:0101090000F5
:01010A0000F4
:01010B0000F3
:01010C0000F2
:01010D0000F1
:01010E0000F0
:01010F0000EF
:0101100000EE
:0101110000ED
:0101120000EC
:0101130000EB
:0101140000EA
:0101150000E9
:0101160000E8
:0101170000E7
:0101180000E6
:0101190000E5
:01011A0000E4
:01011B0000E3
:01011C0000E2
:01011D0000E1
:01011E0000E0
:01011F0000DF
:0101200000DE
:0101210000DD
:0101220000DC
:0101230000DB
:0101240000DA
:0101250000D9
:0101260000D8
:0101270000D7
:0101280000D6
:0101290000D5
:01012A0000D4
:01012B0000D3
:01012C0000D2
:01012D0000D1
:01012E0000D0
:01012F0000CF
:0101300000CE
:0101310000CD
:0101320000CC
:0101330000CB
:0101340000CA
:0101350000C9
:0101360000C8
:0101370000C7
:0101380000C6
:0101390000C5
:01013A0000C4
:01013B0000C3
:01013C0000C2
:01013D0000C1
:01013E0000C0
:01013F0000BF
:0101400000BE
:0101410000BD
:0101420000BC
:0101430000BB
:0101440000BA
:0101450000B9
:0101460000B8
:0101470000B7
:0101480000B6
:0101490000B5
:01014A0000B4
:01014B0000B3
:01014C0000B2
:01014D0000B1
:01014E0000B0
:01014F0000AF
:0101500000AE
:0101510000AD
:0101520000AC
:0101530000AB
:0101540000AA
:0101550000A9
:0101560000A8
:0101570000A7
:0101580000A6
:0101590000A5
:01015A0000A4
:01015B0000A3
:01015C0000A2
:01015D0000A1
:01015E0000A0
:01015F00009F
:01016000009E
:01016100009D
:01016200009C
:01016300009B
:01016400009A
:010165000099
:010166000098
:010167000097
:010168000096
:010169000095
:01016A000094
:01016B000093
:01016C000092
:01016D000091
:01016E000090
:01016F00008F
:01017000008E
:01017100008D
:01017200008C
:01017300008B
:01017400008A
:010175000089
:010176000088
:010177000087
:010178000086
:010179000085
:01017A000084
:01017B000083
:01017C000082
:01017D000081
:01017E000080
:01017F00007F
:01018000007E
:01018100007D
:01018200007C
:01018300007B
:01018400007A
:010185000079
:010186000078
:010187000077
:010188000076
:010189000075
:01018A000074
:01018B000073
:01018C000072
:01018D000071
:01018E000070
:01018F00006F
:01019000006E
:01019100006D
:01019200006C
:01019300006B
:01019400006A
:010195000069
:010196000068
:010197000067
:010198000066
:010199000065
:01019A000064
:01019B000063
:01019C000062
:01019D000061
:01019E000060
:01019F00005F
:0101A000005E
:0101A100005D
:0101A200005C
:0101A300005B
:0101A400005A
:0101A5000059
:0101A6000058
:0101A7000057
:0101A8000056
:0101A9000055
:0101AA000054
:0101AB000053
:0101AC000052
:0101AD000051
:0101AE000050
:0101AF00004F
:0101B000004E
:0101B100004D
:0101B200004C
:0101B300004B
:0101B400004A
:0101B5000049
:0101B6000048
:0101B7000047
:0101B8000046
:0101B9000045
:0101BA000044
:0101BB000043
:0101BC000042
:0101BD000041
:0101BE000040
:0101BF00003F
:0101C000003E
:0101C100003D
:0101C200003C
:0101C300003B
:0101C400003A
:0101C5000039
:0101C6000038
:0101C7000037
:0101C8000036
:0101C9000035
:0101CA000034
:0101CB000033
:0101CC000032
:0101CD000031
:0101CE000030
:0101CF00002F
:0101D000002E
:0101D100002D
:0101D200002C
:0101D300002B
:0101D400002A
:0101D5000029
:0101D6000028
:0101D7000027
:0101D8000026
:0101D9000025
:0101DA000024
:0101DB000023
:0101DC000022
:0101DD000021
:0101DE000020
:0101DF00001F
:0101E000001E
:0101E100001D
:0101E200001C
:0101E300001B
:0101E400001A
:0101E5000019
:0101E6000018
:0101E7000017
:0101E8000016
:0101E9000015
:0101EA000014
:0101EB000013
:0101EC000012
:0101ED000011
:0101EE000010
:0101EF00000F
:0101F000000E
:0101F100000D
:0101F200000C
:0101F300000B
:0101F400000A
:0101F5000009
:0101F6000008
:0101F7000007
:0101F8000006
:0101F9000005
:0101FA000004
:0101FB000003
:0101FC000002
:0101FD000001
:0101FE000000
:0101FF0000FF
:0102000000FD
:0102010000FC
:0102020000FB
:0102030000FA
:0102040000F9
:0102050000F8
:0102060000F7
:0102070000F6
:0102080000F5
:0102090000F4
:01020A0000F3
:01020B0000F2
:01020C0000F1
:01020D0000F0
:01020E0000EF
:01020F0000EE
:0102100000ED
:0102110000EC
:0102120000EB
:0102130000EA
:0102140000E9
:0102150000E8
:0102160000E7
:0102170000E6
:0102180000E5
:0102190000E4
:01021A0000E3
:01021B0000E2
:01021C0000E1
:01021D0000E0
:01021E0000DF
:01021F0000DE
:0102200000DD
:0102210000DC
:0102220000DB
:0102230000DA
:0102240000D9
:0102250000D8
:0102260000D7
:0102270000D6
:0102280000D5
:0102290000D4
:01022A0000D3
:01022B0000D2
:01022C0000D1
:01022D0000D0
:01022E0000CF
:01022F0000CE
:0102300000CD
:0102310000CC
:0102320000CB
:0102330000CA
:0102340000C9
:0102350000C8
:0102360000C7
:0102370000C6
:0102380000C5
:0102390000C4
:01023A0000C3
:01023B0000C2
:01023C0000C1
:01023D0000C0
:01023E0000BF
:01023F0000BE
:0102400000BD
:0102410000BC
:0102420000BB
:0102430000BA
:0102440000B9
:0102450000B8
:0102460000B7
:0102470000B6
:0102480000B5
:0102490000B4
:01024A0000B3
:01024B0000B2
:01024C0000B1
:01024D0000B0
:01024E0000AF
:01024F0000AE
:0102500000AD
:0102510000AC
:0102520000AB
:0102530000AA
:0102540000A9
:0102550000A8
:0102560000A7
:0102570000A6
:0102580000A5
:0102590000A4
:01025A0000A3
:01025B0000A2
:01025C0000A1
:01025D0000A0
:01025E00009F
:01025F00009E
:01026000009D
:01026100009C
:01026200009B
:01026300009A
:010264000099
:010265000098
:010266000097
:010267000096
:010268000095
:010269000094
:01026A000093
:01026B000092
:01026C000091
:01026D000090
:01026E00008F
:01026F00008E
:01027000008D
:01027100008C
:01027200008B
:01027300008A
:010274000089
:010275000088
:010276000087
:010277000086
:010278000085
:010279000084
:01027A000083
:01027B000082
:01027C000081
:01027D000080
:01027E00007F
:01027F00007E
:01028000007D
:01028100007C
:01028200007B
:01028300007A
:010284000079
:010285000078
:010286000077
:010287000076
:010288000075
:010289000074
:01028A000073
:01028B000072
:01028C000071
:01028D000070
:01028E00006F
:01028F00006E
:01029000006D
:01029100006C
:01029200006B
:01029300006A
:010294000069
:010295000068
:010296000067
:010297000066
:010298000065
:010299000064
:01029A000063
:01029B000062
:01029C000061
:01029D000060
:01029E00005F
:01029F00005E
:0102A000005D
:0102A100005C
:0102A200005B
:0102A300005A
:0102A4000059
:0102A5000058
:0102A6000057
:0102A7000056
:0102A8000055
:0102A9000054
:0102AA000053
:0102AB000052
:0102AC000051
:0102AD000050
:0102AE00004F
:0102AF00004E
:0102B000004D
:0102B100004C
:0102B200004B
:0102B300004A
:0102B4000049
:0102B5000048
:0102B6000047
:0102B7000046
:0102B8000045
:0102B9000044
:0102BA000043
:0102BB000042
:0102BC000041
:0102BD000040
:0102BE00003F
:0102BF00003E
:0102C000003D
:0102C100003C
:0102C200003B
:0102C300003A
:0102C4000039
:0102C5000038
:0102C6000037
:0102C7000036
:0102C8000035
:0102C9000034
:0102CA000033
:0102CB000032
:0102CC000031
:0102CD000030
:0102CE00002F
:0102CF00002E
:0102D000002D
:0102D100002C
:0102D200002B
:0102D300002A
:0102D4000029
:0102D5000028
:0102D6000027
:0102D7000026
:0102D8000025
:0102D9000024
:0102DA000023
:0102DB000022
:0102DC000021
:0102DD000020
:0102DE00001F
:0102DF00001E
:0102E000001D
:0102E100001C
:0102E200001B
:0102E300001A
:0102E4000019
:0102E5000018
:0102E6000017
:0102E7000016
:0102E8000015
:0102E9000014
:0102EA000013
:0102EB000012
:0102EC000011
:0102ED000010
:0102EE00000F
:0102EF00000E
:0102F000000D
:0102F100000C
:0102F200000B
:0102F300000A
:0102F4000009
:0102F5000008
:0102F6000007
:0102F7000006
:0102F8000005
:0102F9000004
:0102FA000003
:0102FB000002
:0102FC000001
:0102FD000000
:0102FE0000FF
:0102FF0000FE
:0103000000FC
:0103010000FB
:0103020000FA
:0103030000F9
:0103040000F8
:0103050000F7
:0103060000F6
:0103070000F5
:0103080000F4
:0103090000F3
:01030A0000F2
:01030B0000F1
:01030C0000F0
:01030D0000EF
:01030E0000EE
:01030F0000ED
:0103100000EC
:0103110000EB
:0103120000EA
:0103130000E9
:0103140000E8
:0103150000E7
:0103160000E6
:0103170000E5
:0103180000E4
:0103190000E3
:01031A0000E2
:01031B0000E1
:01031C0000E0
:01031D0000DF
:01031E0000DE
:01031F0000DD
:0103200000DC
:0103210000DB
:0103220000DA
:0103230000D9
:0103240000D8
:0103250000D7
:0103260000D6
:0103270000D5
:0103280000D4
:0103290000D3
:01032A0000D2
:01032B0000D1
:01032C0000D0
:01032D0000CF
:01032E0000CE
:01032F0000CD
:0103300000CC
:0103310000CB
:0103320000CA
:0103330000C9
:0103340000C8
:0103350000C7
:0103360000C6
:0103370000C5
:0103380000C4
:0103390000C3
:01033A0000C2
:01033B0000C1
:01033C0000C0
:01033D0000BF
:01033E0000BE
:01033F0000BD
:0103400000BC
:0103410000BB
:0103420000BA
:0103430000B9
:0103440000B8
:0103450000B7
:0103460000B6
:0103470000B5
:0103480000B4
:0103490000B3
:01034A0000B2
:01034B0000B1
:01034C0000B0
:01034D0000AF
:01034E0000AE
:01034F0000AD
:0103500000AC
:0103510000AB
:0103520000AA
:0103530000A9
:0103540000A8
:0103550000A7
:0103560000A6
:0103570000A5
:0103580000A4
:0103590000A3
:01035A0000A2
:01035B0000A1
:01035C0000A0
:01035D00009F
:01035E00009E
:01035F00009D
:01036000009C
:01036100009B
:01036200009A
:010363000099
:010364000098
:010365000097
:010366000096
:010367000095
:010368000094
:010369000093
:01036A000092
:01036B000091
:01036C000090
:01036D00008F
:01036E00008E
:01036F00008D
:01037000008C
:01037100008B
:01037200008A
:010373000089
:010374000088
:010375000087
:010376000086
:010377000085
:010378000084
:010379000083
:01037A000082
:01037B000081
:01037C000080
:01037D00007F
:01037E00007E
:01037F00007D
:01038000007C
:01038100007B
:01038200007A
:010383000079
:010384000078
:010385000077
:010386000076
:010387000075
:010388000074
:010389000073
:01038A000072
:01038B000071
:01038C000070
:01038D00006F
:01038E00006E
:01038F00006D
:01039000006C
:01039100006B
:01039200006A
:010393000069
:010394000068
:010395000067
:010396000066
:010397000065
:010398000064
:010399000063
:01039A000062
:01039B000061
:01039C000060
:01039D00005F
:01039E00005E
:01039F00005D
:0103A000005C
:0103A100005B
:0103A200005A
:0103A3000059
:0103A4000058
:0103A5000057
:0103A6000056
:0103A7000055
:0103A8000054
:0103A9000053
:0103AA000052
:0103AB000051
:0103AC000050
:0103AD00004F
:0103AE00004E
:0103AF00004D
:0103B000004C
:0103B100004B
:0103B200004A
:0103B3000049
:0103B4000048
:0103B5000047
:0103B6000046
:0103B7000045
:0103B8000044
:0103B9000043
:0103BA000042
:0103BB000041
:0103BC000040
:0103BD00003F
:0103BE00003E
:0103BF00003D
:0103C000003C
:0103C100003B
:0103C200003A
:0103C3000039
:0103C4000038
:0103C5000037
:0103C6000036
:0103C7000035
:0103C8000034
:0103C9000033
:0103CA000032
:0103CB000031
:0103CC000030
:0103CD00002F
:0103CE00002E
:0103CF00002D
:0103D000002C
:0103D100002B
:0103D200002A
:0103D3000029
:0103D4000028
:0103D5000027
:0103D6000026
:0103D7000025
:0103D8000024
:0103D9000023
:0103DA000022
:0103DB000021
:0103DC000020
:0103DD00001F
:0103DE00001E
:0103DF00001D
:0103E000001C
:0103E100001B
:0103E200001A
:0103E3000019
:0103E4000018
:0103E5000017
:0103E6000016
:0103E7000015
:0103E8000014
:0103E9000013
:0103EA000012
:0103EB000011
:0103EC000010
:0103ED00000F
:0103EE00000E
:0103EF00000D
:0103F000000C
:0103F100000B
:0103F200000A
:0103F3000009
:0103F4000008
:0103F5000007
:0103F6000006
:0103F7000005
:0103F8000004
:0103F9000003
:0103FA000002
:0103FB000001
:0103FC000000
:0103FD0000FF
:0103FE0000FE
:0103FF0000FD
:0104000000FB
:0104010000FA
:0104020000F9
:0104030000F8
:0104040000F7
:0104050000F6
:0104060000F5
:0104070000F4
:0104080000F3
:0104090000F2
:01040A0000F1
:01040B0000F0
:01040C0000EF
:01040D0000EE
:01040E0000ED
:01040F0000EC
:0104100000EB
:0104110000EA
:0104120000E9
:0104130000E8
:0104140000E7
:0104150000E6
:0104160000E5
:0104170000E4
:0104180000E3
:0104190000E2
:01041A0000E1
:01041B0000E0
:01041C0000DF
:01041D0000DE
:01041E0000DD
:01041F0000DC
:0104200000DB
:0104210000DA
:0104220000D9
:0104230000D8
:0104240000D7
:0104250000D6
:0104260000D5
:0104270000D4
:0104280000D3
:0104290000D2
:01042A0000D1
:01042B0000D0
:01042C0000CF
:01042D0000CE
:01042E0000CD
:01042F0000CC
:0104300000CB
:0104310000CA
:0104320000C9
:0104330000C8
:0104340000C7
:0104350000C6
:0104360000C5
:0104370000C4
:0104380000C3
:0104390000C2
:01043A0000C1
:01043B0000C0
:01043C0000BF
:01043D0000BE
:01043E0000BD
:01043F0000BC
:0104400000BB
:0104410000BA
:0104420000B9
:0104430000B8
:0104440000B7
:0104450000B6
:0104460000B5
:0104470000B4
:0104480000B3
:0104490000B2
:01044A0000B1
:01044B0000B0
:01044C0000AF
:01044D0000AE
:01044E0000AD
:01044F0000AC
:0104500000AB
:0104510000AA
:0104520000A9
:0104530000A8
:0104540000A7
:0104550000A6
:0104560000A5
:0104570000A4
:0104580000A3
:0104590000A2
:01045A0000A1
:01045B0000A0
:01045C00009F
:01045D00009E
:01045E00009D
:01045F00009C
:01046000009B
:01046100009A
:010462000099
:010463000098
:010464000097
:010465000096
:010466000095
:010467000094
:010468000093
:010469000092
:01046A000091
:01046B000090
:01046C00008F
:01046D00008E
:01046E00008D
:01046F00008C
:01047000008B
:01047100008A
:010472000089
:010473000088
:010474000087
:010475000086
:010476000085
:010477000084
:010478000083
:010479000082
:01047A000081
:01047B000080
:01047C00007F
:01047D00007E
:01047E00007D
:01047F00007C
:01048000007B
:01048100007A
:010482000079
:010483000078
:010484000077
:010485000076
:010486000075
:010487000074
:010488000073
:010489000072
:01048A000071
:01048B000070
:01048C00006F
:01048D00006E
:01048E00006D
:01048F00006C
:01049000006B
:01049100006A
:010492000069
:010493000068
:010494000067
:010495000066
:010496000065
:010497000064
:010498000063
:010499000062
:01049A000061
:01049B000060
:01049C00005F
:01049D00005E
:01049E00005D
:01049F00005C
:0104A000005B
:0104A100005A
:0104A2000059
:0104A3000058
:0104A4000057
:0104A5000056
:0104A6000055
:0104A7000054
:0104A8000053
:0104A9000052
:0104AA000051
:0104AB000050
:0104AC00004F
:0104AD00004E
:0104AE00004D
:0104AF00004C
:0104B000004B
:0104B100004A
:0104B2000049
:0104B3000048
:0104B4000047
:0104B5000046
:0104B6000045
:0104B7000044
:0104B8000043
:0104B9000042
:0104BA000041
:0104BB000040
:0104BC00003F
:0104BD00003E
:0104BE00003D
:0104BF00003C
:0104C000003B
:0104C100003A
:0104C2000039
:0104C3000038
:0104C4000037
:0104C5000036
:0104C6000035
:0104C7000034
:0104C8000033
:0104C9000032
:0104CA000031
:0104CB000030
:0104CC00002F
:0104CD00002E
:0104CE00002D
:0104CF00002C
:0104D000002B
:0104D100002A
:0104D2000029
:0104D3000028
:0104D4000027
:0104D5000026
:0104D6000025
:0104D7000024
:0104D8000023
:0104D9000022
:0104DA000021
:0104DB000020
:0104DC00001F
:0104DD00001E
:0104DE00001D
:0104DF00001C
:0104E000001B
:0104E100001A
:0104E2000019
:0104E3000018
:0104E4000017
:0104E5000016
:0104E6000015
:0104E7000014
:0104E8000013
:0104E9000012
:0104EA000011
:0104EB000010
:0104EC00000F
:0104ED00000E
:0104EE00000D
:0104EF00000C
:0104F000000B
:0104F100000A
:0104F2000009
:0104F3000008
:0104F4000007
:0104F5000006
:0104F6000005
:0104F7000004
:0104F8000003
:0104F9000002
:0104FA000001
:0104FB000000
:0104FC0000FF
:0104FD0000FE
:0104FE0000FD
:0104FF0000FC
:0105000000FA
:0105010000F9
:0105020000F8
:0105030000F7
:0105040000F6
:0105050000F5
:0105060000F4
:0105070000F3
:0105080000F2
:0105090000F1
:01050A0000F0
:01050B0000EF
:01050C0000EE
:01050D0000ED
:01050E0000EC
:01050F0000EB
:0105100000EA
:0105110000E9
:0105120000E8
:0105130000E7
:0105140000E6
:0105150000E5
:0105160000E4
:0105170000E3
:0105180000E2
:0105190000E1
:01051A0000E0
:01051B0000DF
:01051C0000DE
:01051D0000DD
:01051E0000DC
:01051F0000DB
:0105200000DA
:0105210000D9
:0105220000D8
:0105230000D7
:0105240000D6
:0105250000D5
:0105260000D4
:0105270000D3
:0105280000D2
:0105290000D1
:01052A0000D0
:01052B0000CF
:01052C0000CE
:01052D0000CD
:01052E0000CC
:01052F0000CB
:0105300000CA
:0105310000C9
:0105320000C8
:0105330000C7
:0105340000C6
:0105350000C5
:0105360000C4
:0105370000C3
:0105380000C2
:0105390000C1
:01053A0000C0
:01053B0000BF
:01053C0000BE
:01053D0000BD
:01053E0000BC
:01053F0000BB
:0105400000BA
:0105410000B9
:0105420000B8
:0105430000B7
:0105440000B6
:0105450000B5
:0105460000B4
:0105470000B3
:0105480000B2
:0105490000B1
:01054A0000B0
:01054B0000AF
:01054C0000AE
:01054D0000AD
:01054E0000AC
:01054F0000AB
:0105500000AA
:0105510000A9
:0105520000A8
:0105530000A7
:0105540000A6
:0105550000A5
:0105560000A4
:0105570000A3
:0105580000A2
:0105590000A1
:01055A0000A0
:01055B00009F
:01055C00009E
:01055D00009D
:01055E00009C
:01055F00009B
:01056000009A
:010561000099
:010562000098
:010563000097
:010564000096
:010565000095
:010566000094
:010567000093
:010568000092
:010569000091
:01056A000090
:01056B00008F
:01056C00008E
:01056D00008D
:01056E00008C
:01056F00008B
:01057000008A
:010571000089
:010572000088
:010573000087
:010574000086
:010575000085
:010576000084
:010577000083
:010578000082
:010579000081
:01057A000080
:01057B00007F
:01057C00007E
:01057D00007D
:01057E00007C
:01057F00007B
:01058000007A
:010581000079
:010582000078
:010583000077
:010584000076
:010585000075
:010586000074
:010587000073
:010588000072
:010589000071
:01058A000070
:01058B00006F
:01058C00006E
:01058D00006D
:01058E00006C
:01058F00006B
:01059000006A
:010591000069
:010592000068
:010593000067
:010594000066
:010595000065
:010596000064
:010597000063
:010598000062
:010599000061
:01059A000060
:01059B00005F
:01059C00005E
:01059D00005D
:01059E00005C
:01059F00005B
:0105A000005A
:0105A1000059
:0105A2000058
:0105A3000057
:0105A4000056
:0105A5000055
:0105A6000054
:0105A7000053
:0105A8000052
:0105A9000051
:0105AA000050
:0105AB00004F
:0105AC00004E
:0105AD00004D
:0105AE00004C
:0105AF00004B
:0105B000004A
:0105B1000049
:0105B2000048
:0105B3000047
:0105B4000046
:0105B5000045
:0105B6000044
:0105B7000043
:0105B8000042
:0105B9000041
:0105BA000040
:0105BB00003F
:0105BC00003E
:0105BD00003D
:0105BE00003C
:0105BF00003B
:0105C000003A
:0105C1000039
:0105C2000038
:0105C3000037
:0105C4000036
:0105C5000035
:0105C6000034
:0105C7000033
:0105C8000032
:0105C9000031
:0105CA000030
:0105CB00002F
:0105CC00002E
:0105CD00002D
:0105CE00002C
:0105CF00002B
:0105D000002A
:0105D1000029
:0105D2000028
:0105D3000027
:0105D4000026
:0105D5000025
:0105D6000024
:0105D7000023
:0105D8000022
:0105D9000021
:0105DA000020
:0105DB00001F
:0105DC00001E
:0105DD00001D
:0105DE00001C
:0105DF00001B
:0105E000001A
:0105E1000019
:0105E2000018
:0105E3000017
:0105E4000016
:0105E5000015
:0105E6000014
:0105E7000013
:0105E8000012
:0105E9000011
:0105EA000010
:0105EB00000F
:0105EC00000E
:0105ED00000D
:0105EE00000C
:0105EF00000B
:0105F000000A
:0105F1000009
:0105F2000008
:0105F3000007
:0105F4000006
:0105F5000005
:0105F6000004
:0105F7000003
:0105F8000002
:0105F9000001
:0105FA000000
:0105FB0000FF
:0105FC0000FE
:0105FD0000FD
:0105FE0000FC
:0105FF0000FB
:0106000000F9
:0106010000F8
:0106020000F7
:0106030000F6
:0106040000F5
:0106050000F4
:0106060000F3
:0106070000F2
:0106080000F1
:0106090000F0
:01060A0000EF
:01060B0000EE
:01060C0000ED
:01060D0000EC
:01060E0000EB
:01060F0000EA
:0106100000E9
:0106110000E8
:0106120000E7
:0106130000E6
:0106140000E5
:0106150000E4
:0106160000E3
:0106170000E2
:0106180000E1
:0106190000E0
:01061A0000DF
:01061B0000DE
:01061C0000DD
:01061D0000DC
:01061E0000DB
:01061F0000DA
:0106200000D9
:0106210000D8
:0106220000D7
:0106230000D6
:0106240000D5
:0106250000D4
:0106260000D3
:0106270000D2
:0106280000D1
:0106290000D0
:01062A0000CF
:01062B0000CE
:01062C0000CD
:01062D0000CC
:01062E0000CB
:01062F0000CA
:0106300000C9
:0106310000C8
:0106320000C7
:0106330000C6
:0106340000C5
:0106350000C4
:0106360000C3
:0106370000C2
:0106380000C1
:0106390000C0
:01063A0000BF
:01063B0000BE
:01063C0000BD
:01063D0000BC
:01063E0000BB
:01063F0000BA
:0106400000B9
:0106410000B8
:0106420000B7
:0106430000B6
:0106440000B5
:0106450000B4
:0106460000B3
:0106470000B2
:0106480000B1
:0106490000B0
:01064A0000AF
:01064B0000AE
:01064C0000AD
:01064D0000AC
:01064E0000AB
:01064F0000AA
:0106500000A9
:0106510000A8
:0106520000A7
:0106530000A6
:0106540000A5
:0106550000A4
:0106560000A3
:0106570000A2
:0106580000A1
:0106590000A0
:01065A00009F
:01065B00009E
:01065C00009D
:01065D00009C
:01065E00009B
:01065F00009A
:010660000099
:010661000098
:010662000097
:010663000096
:010664000095
:010665000094
:010666000093
:010667000092
:010668000091
:010669000090
:01066A00008F
:01066B00008E
:01066C00008D
:01066D00008C
:01066E00008B
:01066F00008A
:010670000089
:010671000088
:010672000087
:010673000086
:010674000085
:010675000084
:010676000083
:010677000082
:010678000081
:010679000080
:01067A00007F
:01067B00007E
:01067C00007D
:01067D00007C
:01067E00007B
:01067F00007A
:010680000079
:010681000078
:010682000077
:010683000076
:010684000075
:010685000074
:010686000073
:010687000072
:010688000071
:010689000070
:01068A00006F
:01068B00006E
:01068C00006D
:01068D00006C
:01068E00006B
:01068F00006A
:010690000069
:010691000068
:010692000067
:010693000066
:010694000065
:010695000064
:010696000063
:010697000062
:010698000061
:010699000060
:01069A00005F
:01069B00005E
:01069C00005D
:01069D00005C
:01069E00005B
:01069F00005A
:0106A0000059
:0106A1000058
:0106A2000057
:0106A3000056
:0106A4000055
:0106A5000054
:0106A6000053
:0106A7000052
:0106A8000051
:0106A9000050
:0106AA00004F
:0106AB00004E
:0106AC00004D
:0106AD00004C
:0106AE00004B
:0106AF00004A
:0106B0000049
:0106B1000048
:0106B2000047
:0106B3000046
:0106B4000045
:0106B5000044
:0106B6000043
:0106B7000042
:0106B8000041
:0106B9000040
:0106BA00003F
:0106BB00003E
:0106BC00003D
:0106BD00003C
:0106BE00003B
:0106BF00003A
:0106C0000039
:0106C1000038
:0106C2000037
:0106C3000036
:0106C4000035
:0106C5000034
:0106C6000033
:0106C7000032
:0106C8000031
:0106C9000030
:0106CA00002F
:0106CB00002E
:0106CC00002D
:0106CD00002C
:0106CE00002B
:0106CF00002A
:0106D0000029
:0106D1000028
:0106D2000027
:0106D3000026
:0106D4000025
:0106D5000024
:0106D6000023
:0106D7000022
:0106D8000021
:0106D9000020
:0106DA00001F
:0106DB00001E
:0106DC00001D
:0106DD00001C
:0106DE00001B
:0106DF00001A
:0106E0000019
:0106E1000018
:0106E2000017
:0106E3000016
:0106E4000015
:0106E5000014
:0106E6000013
:0106E7000012
:0106E8000011
:0106E9000010
:0106EA00000F
:0106EB00000E
:0106EC00000D
:0106ED00000C
:0106EE00000B
:0106EF00000A
:0106F0000009
:0106F1000008
:0106F2000007
:0106F3000006
:0106F4000005
:0106F5000004
:0106F6000003
:0106F7000002
:0106F8000001
:0106F9000000
:0106FA0000FF
:0106FB0000FE
:0106FC0000FD
:0106FD0000FC
:0106FE0000FB
:0106FF0000FA
:0107000000F8
:0107010000F7
:0107020000F6
:0107030000F5
:0107040000F4
:0107050000F3
:0107060000F2
:0107070000F1
:0107080000F0
:0107090000EF
:01070A0000EE
:01070B0000ED
:01070C0000EC
:01070D0000EB
:01070E0000EA
:01070F0000E9
:0107100000E8
:0107110000E7
:0107120000E6
:0107130000E5
:0107140000E4
:0107150000E3
:0107160000E2
:0107170000E1
:0107180000E0
:0107190000DF
:01071A0000DE
:01071B0000DD
:01071C0000DC
:01071D0000DB
:01071E0000DA
:01071F0000D9
:0107200000D8
:0107210000D7
:0107220000D6
:0107230000D5
:0107240000D4
:0107250000D3
:0107260000D2
:0107270000D1
:0107280000D0
:0107290000CF
:01072A0000CE
:01072B0000CD
:01072C0000CC
:01072D0000CB
:01072E0000CA
:01072F0000C9
:0107300000C8
:0107310000C7
:0107320000C6
:0107330000C5
:0107340000C4
:0107350000C3
:0107360000C2
:0107370000C1
:0107380000C0
:0107390000BF
:01073A0000BE
:01073B0000BD
:01073C0000BC
:01073D0000BB
:01073E0000BA
:01073F0000B9
:0107400000B8
:0107410000B7
:0107420000B6
:0107430000B5
:0107440000B4
:0107450000B3
:0107460000B2
:0107470000B1
:0107480000B0
:0107490000AF
:01074A0000AE
:01074B0000AD
:01074C0000AC
:01074D0000AB
:01074E0000AA
:01074F0000A9
:0107500000A8
:0107510000A7
:0107520000A6
:0107530000A5
:0107540000A4
:0107550000A3
:0107560000A2
:0107570000A1
:0107580000A0
:01075900009F
:01075A00009E
:01075B00009D
:01075C00009C
:01075D00009B
:01075E00009A
:01075F000099
:010760000098
:010761000097
:010762000096
:010763000095
:010764000094
:010765000093
:010766000092
:010767000091
:010768000090
:01076900008F
:01076A00008E
:01076B00008D
:01076C00008C
:01076D00008B
:01076E00008A
:01076F000089
:010770000088
:010771000087
:010772000086
:010773000085
:010774000084
:010775000083
:010776000082
:010777000081
:010778000080
:01077900007F
:01077A00007E
:01077B00007D
:01077C00007C
:01077D00007B
:01077E00007A
:01077F000079
:010780000078
:010781000077
:010782000076
:010783000075
:010784000074
:010785000073
:010786000072
:010787000071
:010788000070
:01078900006F
:01078A00006E
:01078B00006D
:01078C00006C
:01078D00006B
:01078E00006A
:01078F000069
:010790000068
:010791000067
:010792000066
:010793000065
:010794000064
:010795000063
:010796000062
:010797000061
:010798000060
:01079900005F
:01079A00005E
:01079B00005D
:01079C00005C
:01079D00005B
:01079E00005A
:01079F000059
:0107A0000058
:0107A1000057
:0107A2000056
:0107A3000055
:0107A4000054
:0107A5000053
:0107A6000052
:0107A7000051
:0107A8000050
:0107A900004F
:0107AA00004E
:0107AB00004D
:0107AC00004C
:0107AD00004B
:0107AE00004A
:0107AF000049
:0107B0000048
:0107B1000047
:0107B2000046
:0107B3000045
:0107B4000044
:0107B5000043
:0107B6000042
:0107B7000041
:0107B8000040
:0107B900003F
:0107BA00003E
:0107BB00003D
:0107BC00003C
:0107BD00003B
:0107BE00003A
:0107BF000039
:0107C0000038
:0107C1000037
:0107C2000036
:0107C3000035
:0107C4000034
:0107C5000033
:0107C6000032
:0107C7000031
:0107C8000030
:0107C900002F
:0107CA00002E
:0107CB00002D
:0107CC00002C
:0107CD00002B
:0107CE00002A
:0107CF000029
:0107D0000028
:0107D1000027
:0107D2000026
:0107D3000025
:0107D4000024
:0107D5000023
:0107D6000022
:0107D7000021
:0107D8000020
:0107D900001F
:0107DA00001E
:0107DB00001D
:0107DC00001C
:0107DD00001B
:0107DE00001A
:0107DF000019
:0107E0000018
:0107E1000017
:0107E2000016
:0107E3000015
:0107E4000014
:0107E5000013
:0107E6000012
:0107E7000011
:0107E8000010
:0107E900000F
:0107EA00000E
:0107EB00000D
:0107EC00000C
:0107ED00000B
:0107EE00000A
:0107EF000009
:0107F0000008
:0107F1000007
:0107F2000006
:0107F3000005
:0107F4000004
:0107F5000003
:0107F6000002
:0107F7000001
:0107F8000000
:0107F90000FF
:0107FA0000FE
:0107FB0000FD
:0107FC0000FC
:0107FD0000FB
:0107FE0000FA
:0107FF0000F9
:0108000000F7
:0108010000F6
:0108020000F5
:0108030000F4
:0108040000F3
:0108050000F2
:0108060000F1
:0108070000F0
:0108080000EF
:0108090000EE
:01080A0000ED
:01080B0000EC
:01080C0000EB
:01080D0000EA
:01080E0000E9
:01080F0000E8
:0108100000E7
:0108110000E6
:0108120000E5
:0108130000E4
:0108140000E3
:0108150000E2
:0108160000E1
:0108170000E0
:0108180000DF
:0108190000DE
:01081A0000DD
:01081B0000DC
:01081C0000DB
:01081D0000DA
:01081E0000D9
:01081F0000D8
:0108200000D7
:0108210000D6
:0108220000D5
:0108230000D4
:0108240000D3
:0108250000D2
:0108260000D1
:0108270000D0
:0108280000CF
:0108290000CE
:01082A0000CD
:01082B0000CC
:01082C0000CB
:01082D0000CA
:01082E0000C9
:01082F0000C8
:0108300000C7
:0108310000C6
:0108320000C5
:0108330000C4
:0108340000C3
:0108350000C2
:0108360000C1
:0108370000C0
:0108380000BF
:0108390000BE
:01083A0000BD
:01083B0000BC
:01083C0000BB
:01083D0000BA
:01083E0000B9
:01083F0000B8
:0108400000B7
:0108410000B6
:0108420000B5
:0108430000B4
:0108440000B3
:0108450000B2
:0108460000B1
:0108470000B0
:0108480000AF
:0108490000AE
:01084A0000AD
:01084B0000AC
:01084C0000AB
:01084D0000AA
:01084E0000A9
:01084F0000A8
:0108500000A7
:0108510000A6
:0108520000A5
:0108530000A4
:0108540000A3
:0108550000A2
:0108560000A1
:0108570000A0
:01085800009F
:01085900009E
:01085A00009D
:01085B00009C
:01085C00009B
:01085D00009A
:01085E000099
:01085F000098
:010860000097
:010861000096
:010862000095
:010863000094
:010864000093
:010865000092
:010866000091
:010867000090
:01086800008F
:01086900008E
:01086A00008D
:01086B00008C
:01086C00008B
:01086D00008A
:01086E000089
:01086F000088
:010870000087
:010871000086
:010872000085
:010873000084
:010874000083
:010875000082
:010876000081
:010877000080
:01087800007F
:01087900007E
:01087A00007D
:01087B00007C
:01087C00007B
:01087D00007A
:01087E000079
:01087F000078
:010880000077
:010881000076
:010882000075
:010883000074
:010884000073
:010885000072
:010886000071
:010887000070
:01088800006F
:01088900006E
:01088A00006D
:01088B00006C
:01088C00006B
:01088D00006A
:01088E000069
:01088F000068
:010890000067
:010891000066
:010892000065
:010893000064
:010894000063
:010895000062
:010896000061
:010897000060
:01089800005F
:01089900005E
:01089A00005D
:01089B00005C
:01089C00005B
:01089D00005A
:01089E000059
:01089F000058
:0108A0000057
:0108A1000056
:0108A2000055
:0108A3000054
:0108A4000053
:0108A5000052
:0108A6000051
:0108A7000050
:0108A800004F
:0108A900004E
:0108AA00004D
:0108AB00004C
:0108AC00004B
:0108AD00004A
:0108AE000049
:0108AF000048
:0108B0000047
:0108B1000046
:0108B2000045
:0108B3000044
:0108B4000043
:0108B5000042
:0108B6000041
:0108B7000040
:0108B800003F
:0108B900003E
:0108BA00003D
:0108BB00003C
:0108BC00003B
:0108BD00003A
:0108BE000039
:0108BF000038
:0108C0000037
:0108C1000036
:0108C2000035
:0108C3000034
:0108C4000033
:0108C5000032
:0108C6000031
:0108C7000030
:0108C800002F
:0108C900002E
:0108CA00002D
:0108CB00002C
:0108CC00002B
:0108CD00002A
:0108CE000029
:0108CF000028
:0108D0000027
:0108D1000026
:0108D2000025
:0108D3000024
:0108D4000023
:0108D5000022
:0108D6000021
:0108D7000020
:0108D800001F
:0108D900001E
:0108DA00001D
:0108DB00001C
:0108DC00001B
:0108DD00001A
:0108DE000019
:0108DF000018
:0108E0000017
:0108E1000016
:0108E2000015
:0108E3000014
:0108E4000013
:0108E5000012
:0108E6000011
:0108E7000010
:0108E800000F
:0108E900000E
:0108EA00000D
:0108EB00000C
:0108EC00000B
:0108ED00000A
:0108EE000009
:0108EF000008
:0108F0000007
:0108F1000006
:0108F2000005
:0108F3000004
:0108F4000003
:0108F5000002
:0108F6000001
:0108F7000000
:0108F80000FF
:0108F90000FE
:0108FA0000FD
:0108FB0000FC
:0108FC0000FB
:0108FD0000FA
:0108FE0000F9
:0108FF0000F8
:0109000000F6
:0109010000F5
:0109020000F4
:0109030000F3
:0109040000F2
:0109050000F1
:0109060000F0
:0109070000EF
:0109080000EE
:0109090000ED
:01090A0000EC
:01090B0000EB
:01090C0000EA
:01090D0000E9
:01090E0000E8
:01090F0000E7
:0109100000E6
:0109110000E5
:0109120000E4
:0109130000E3
:0109140000E2
:0109150000E1
:0109160000E0
:0109170000DF
:0109180000DE
:0109190000DD
:01091A0000DC
:01091B0000DB
:01091C0000DA
:01091D0000D9
:01091E0000D8
:01091F0000D7
:0109200000D6
:0109210000D5
:0109220000D4
:0109230000D3
:0109240000D2
:0109250000D1
:0109260000D0
:0109270000CF
:0109280000CE
:0109290000CD
:01092A0000CC
:01092B0000CB
:01092C0000CA
:01092D0000C9
:01092E0000C8
:01092F0000C7
:0109300000C6
:0109310000C5
:0109320000C4
:0109330000C3
:0109340000C2
:0109350000C1
:0109360000C0
:0109370000BF
:0109380000BE
:0109390000BD
:01093A0000BC
:01093B0000BB
:01093C0000BA
:01093D0000B9
:01093E0000B8
:01093F0000B7
:0109400000B6
:0109410000B5
:0109420000B4
:0109430000B3
:0109440000B2
:0109450000B1
:0109460000B0
:0109470000AF
:0109480000AE
:0109490000AD
:01094A0000AC
:01094B0000AB
:01094C0000AA
:01094D0000A9
:01094E0000A8
:01094F0000A7
:0109500000A6
:0109510000A5
:0109520000A4
:0109530000A3
:0109540000A2
:0109550000A1
:0109560000A0
:01095700009F
:01095800009E
:01095900009D
:01095A00009C
:01095B00009B
:01095C00009A
:01095D000099
:01095E000098
:01095F000097
:010960000096
:010961000095
:010962000094
:010963000093
:010964000092
:010965000091
:010966000090
:01096700008F
:01096800008E
:01096900008D
:01096A00008C
:01096B00008B
:01096C00008A
:01096D000089
:01096E000088
:01096F000087
:010970000086
:010971000085
:010972000084
:010973000083
:010974000082
:010975000081
:010976000080
:01097700007F
:01097800007E
:01097900007D
:01097A00007C
:01097B00007B
:01097C00007A
:01097D000079
:01097E000078
:01097F000077
:010980000076
:010981000075
:010982000074
:010983000073
:010984000072
:010985000071
:010986000070
:01098700006F
:01098800006E
:01098900006D
:01098A00006C
:01098B00006B
:01098C00006A
:01098D000069
:01098E000068
:01098F000067
:010990000066
:010991000065
:010992000064
:010993000063
:010994000062
:010995000061
:010996000060
:01099700005F
:01099800005E
:01099900005D
:01099A00005C
:01099B00005B
:01099C00005A
:01099D000059
:01099E000058
:01099F000057
:0109A0000056
:0109A1000055
:0109A2000054
:0109A3000053
:0109A4000052
:0109A5000051
:0109A6000050
:0109A700004F
:0109A800004E
:0109A900004D
:0109AA00004C
:0109AB00004B
:0109AC00004A
:0109AD000049
:0109AE000048
:0109AF000047
:0109B0000046
:0109B1000045
:0109B2000044
:0109B3000043
:0109B4000042
:0109B5000041
:0109B6000040
:0109B700003F
:0109B800003E
:0109B900003D
:0109BA00003C
:0109BB00003B
:0109BC00003A
:0109BD000039
:0109BE000038
:0109BF000037
:0109C0000036
:0109C1000035
:0109C2000034
:0109C3000033
:0109C4000032
:0109C5000031
:0109C6000030
:0109C700002F
:0109C800002E
:0109C900002D
:0109CA00002C
:0109CB00002B
:0109CC00002A
:0109CD000029
:0109CE000028
:0109CF000027
:0109D0000026
:0109D1000025
:0109D2000024
:0109D3000023
:0109D4000022
:0109D5000021
:0109D6000020
:0109D700001F
:0109D800001E
:0109D900001D
:0109DA00001C
:0109DB00001B
:0109DC00001A
:0109DD000019
:0109DE000018
:0109DF000017
:0109E0000016
:0109E1000015
:0109E2000014
:0109E3000013
:0109E4000012
:0109E5000011
:0109E6000010
:0109E700000F
:0109E800000E
:0109E900000D
:0109EA00000C
:0109EB00000B
:0109EC00000A
:0109ED000009
:0109EE000008
:0109EF000007
:0109F0000006
:0109F1000005
:0109F2000004
:0109F3000003
:0109F4000002
:0109F5000001
:0109F6000000
:0109F70000FF
:0109F80000FE
:0109F90000FD
:0109FA0000FC
:0109FB0000FB
:0109FC0000FA
:0109FD0000F9
:0109FE0000F8
:0109FF0000F7
:010A000000F5
:010A010000F4
:010A020000F3
:010A030000F2
:010A040000F1
:010A050000F0
:010A060000EF
:010A070000EE
:010A080000ED
:010A090000EC
:010A0A0000EB
:010A0B0000EA
:010A0C0000E9
:010A0D0000E8
:010A0E0000E7
:010A0F0000E6
:010A100000E5
:010A110000E4
:010A120000E3
:010A130000E2
:010A140000E1
:010A150000E0
:010A160000DF
:010A170000DE
:010A180000DD
:010A190000DC
:010A1A0000DB
:010A1B0000DA
:010A1C0000D9
:010A1D0000D8
:010A1E0000D7
:010A1F0000D6
:010A200000D5
:010A210000D4
:010A220000D3
:010A230000D2
:010A240000D1
:010A250000D0
:010A260000CF
:010A270000CE
:010A280000CD
:010A290000CC
:010A2A0000CB
:010A2B0000CA
:010A2C0000C9
:010A2D0000C8
:010A2E0000C7
:010A2F0000C6
:010A300000C5
:010A310000C4
:010A320000C3
:010A330000C2
:010A340000C1
:010A350000C0
:010A360000BF
:010A370000BE
:010A380000BD
:010A390000BC
:010A3A0000BB
:010A3B0000BA
:010A3C0000B9
:010A3D0000B8
:010A3E0000B7
:010A3F0000B6
:010A400000B5
:010A410000B4
:010A420000B3
:010A430000B2
:010A440000B1
:010A450000B0
:010A460000AF
:010A470000AE
:010A480000AD
:010A490000AC
:010A4A0000AB
:010A4B0000AA
:010A4C0000A9
:010A4D0000A8
:010A4E0000A7
:010A4F0000A6
:010A500000A5
:010A510000A4
:010A520000A3
:010A530000A2
:010A540000A1
:010A550000A0
:010A5600009F
:010A5700009E
:010A5800009D
:010A5900009C
:010A5A00009B
:010A5B00009A
:010A5C000099
:010A5D000098
:010A5E000097
:010A5F000096
:010A60000095
:010A61000094
:010A62000093
:010A63000092
:010A64000091
:010A65000090
:010A6600008F
:010A6700008E
:010A6800008D
:010A6900008C
:010A6A00008B
:010A6B00008A
:010A6C000089
:010A6D000088
:010A6E000087
:010A6F000086
:010A70000085
:010A71000084
:010A72000083
:010A73000082
:010A74000081
:010A75000080
:010A7600007F
:010A7700007E
:010A7800007D
:010A7900007C
:010A7A00007B
:010A7B00007A
:010A7C000079
:010A7D000078
:010A7E000077
:010A7F000076
:010A80000075
:010A81000074
:010A82000073
:010A83000072
:010A84000071
:010A85000070
:010A8600006F
:010A8700006E
:010A8800006D
:010A8900006C
:010A8A00006B
:010A8B00006A
:010A8C000069
:010A8D000068
:010A8E000067
:010A8F000066
:010A90000065
:010A91000064
:010A92000063
:010A93000062
:010A94000061
:010A95000060
:010A9600005F
:010A9700005E
:010A9800005D
:010A9900005C
:010A9A00005B
:010A9B00005A
:010A9C000059
:010A9D000058
:010A9E000057
:010A9F000056
:010AA0000055
:010AA1000054
:010AA2000053
:010AA3000052
:010AA4000051
:010AA5000050
:010AA600004F
:010AA700004E
:010AA800004D
:010AA900004C
:010AAA00004B
:010AAB00004A
:010AAC000049
:010AAD000048
:010AAE000047
:010AAF000046
:010AB0000045
:010AB1000044
:010AB2000043
:010AB3000042
:010AB4000041
:010AB5000040
:010AB600003F
:010AB700003E
:010AB800003D
:010AB900003C
:010ABA00003B
:010ABB00003A
:010ABC000039
:010ABD000038
:010ABE000037
:010ABF000036
:010AC0000035
:010AC1000034
:010AC2000033
:010AC3000032
:010AC4000031
:010AC5000030
:010AC600002F
:010AC700002E
:010AC800002D
:010AC900002C
:010ACA00002B
:010ACB00002A
:010ACC000029
:010ACD000028
:010ACE000027
:010ACF000026
:010AD0000025
:010AD1000024
:010AD2000023
:010AD3000022
:010AD4000021
:010AD5000020
:010AD600001F
:010AD700001E
:010AD800001D
:010AD900001C
:010ADA00001B
:010ADB00001A
:010ADC000019
:010ADD000018
:010ADE000017
:010ADF000016
:010AE0000015
:010AE1000014
:010AE2000013
:010AE3000012
:010AE4000011
:010AE5000010
:010AE600000F
:010AE700000E
:010AE800000D
:010AE900000C
:010AEA00000B
:010AEB00000A
:010AEC000009
:010AED000008
:010AEE000007
:010AEF000006
:010AF0000005
:010AF1000004
:010AF2000003
:010AF3000002
:010AF4000001
:010AF5000000
:010AF60000FF
:010AF70000FE
:010AF80000FD
:010AF90000FC
:010AFA0000FB
:010AFB0000FA
:010AFC0000F9
:010AFD0000F8
:010AFE0000F7
:010AFF0000F6
:010B000000F4
:010B010000F3
:010B020000F2
:010B030000F1
:010B040000F0
:010B050000EF
:010B060000EE
:010B070000ED
:010B080000EC
:010B090000EB
:010B0A0000EA
:010B0B0000E9
:010B0C0000E8
:010B0D0000E7
:010B0E0000E6
:010B0F0000E5
:010B100000E4
:010B110000E3
:010B120000E2
:010B130000E1
:010B140000E0
:010B150000DF
:010B160000DE
:010B170000DD
:010B180000DC
:010B190000DB
:010B1A0000DA
:010B1B0000D9
:010B1C0000D8
:010B1D0000D7
:010B1E0000D6
:010B1F0000D5
:010B200000D4
:010B210000D3
:010B220000D2
:010B230000D1
:010B240000D0
:010B250000CF
:010B260000CE
:010B270000CD
:010B280000CC
:010B290000CB
:010B2A0000CA
:010B2B0000C9
:010B2C0000C8
:010B2D0000C7
:010B2E0000C6
:010B2F0000C5
:010B300000C4
:010B310000C3
:010B320000C2
:010B330000C1
:010B340000C0
:010B350000BF
:010B360000BE
:010B370000BD
:010B380000BC
:010B390000BB
:010B3A0000BA
:010B3B0000B9
:010B3C0000B8
:010B3D0000B7
:010B3E0000B6
:010B3F0000B5
:010B400000B4
:010B410000B3
:010B420000B2
:010B430000B1
:010B440000B0
:010B450000AF
:010B460000AE
:010B470000AD
:010B480000AC
:010B490000AB
:010B4A0000AA
:010B4B0000A9
:010B4C0000A8
:010B4D0000A7
:010B4E0000A6
:010B4F0000A5
:010B500000A4
:010B510000A3
:010B520000A2
:010B530000A1
:010B540000A0
:010B5500009F
:010B5600009E
:010B5700009D
:010B5800009C
:010B5900009B
:010B5A00009A
:010B5B000099
:010B5C000098
:010B5D000097
:010B5E000096
:010B5F000095
:010B60000094
:010B61000093
:010B62000092
:010B63000091
:010B64000090
:010B6500008F
:010B6600008E
:010B6700008D
:010B6800008C
:010B6900008B
:010B6A00008A
:010B6B000089
:010B6C000088
:010B6D000087
:010B6E000086
:010B6F000085
:010B70000084
:010B71000083
:010B72000082
:010B73000081
:010B74000080
:010B7500007F
:010B7600007E
:010B7700007D
:010B7800007C
:010B7900007B
:010B7A00007A
:010B7B000079
:010B7C000078
:010B7D000077
:010B7E000076
:010B7F000075
:010B80000074
:010B81000073
:010B82000072
:010B83000071
:010B84000070
:010B8500006F
:010B8600006E
:010B8700006D
:010B8800006C
:010B8900006B
:010B8A00006A
:010B8B000069
:010B8C000068
:010B8D000067
:010B8E000066
:010B8F000065
:010B90000064
:010B91000063
:010B92000062
:010B93000061
:010B94000060
:010B9500005F
:010B9600005E
:010B9700005D
:010B9800005C
:010B9900005B
:010B9A00005A
:010B9B000059
:010B9C000058
:010B9D000057
:010B9E000056
:010B9F000055
:010BA0000054
:010BA1000053
:010BA2000052
:010BA3000051
:010BA4000050
:010BA500004F
:010BA600004E
:010BA700004D
:010BA800004C
:010BA900004B
:010BAA00004A
:010BAB000049
:010BAC000048
:010BAD000047
:010BAE000046
:010BAF000045
:010BB0000044
:010BB1000043
:010BB2000042
:010BB3000041
:010BB4000040
:010BB500003F
:010BB600003E
:010BB700003D
:010BB800003C
:010BB900003B
:010BBA00003A
:010BBB000039
:010BBC000038
:010BBD000037
:010BBE000036
:010BBF000035
:010BC0000034
:010BC1000033
:010BC2000032
:010BC3000031
:010BC4000030
:010BC500002F
:010BC600002E
:010BC700002D
:010BC800002C
:010BC900002B
:010BCA00002A
:010BCB000029
:010BCC000028
:010BCD000027
:010BCE000026
:010BCF000025
:010BD0000024
:010BD1000023
:010BD2000022
:010BD3000021
:010BD4000020
:010BD500001F
:010BD600001E
:010BD700001D
:010BD800001C
:010BD900001B
:010BDA00001A
:010BDB000019
:010BDC000018
:010BDD000017
:010BDE000016
:010BDF000015
:010BE0000014
:010BE1000013
:010BE2000012
:010BE3000011
:010BE4000010
:010BE500000F
:010BE600000E
:010BE700000D
:010BE800000C
:010BE900000B
:010BEA00000A
:010BEB000009
:010BEC000008
:010BED000007
:010BEE000006
:010BEF000005
:010BF0000004
:010BF1000003
:010BF2000002
:010BF3000001
:010BF4000000
:010BF50000FF
:010BF60000FE
:010BF70000FD
:010BF80000FC
:010BF90000FB
:010BFA0000FA
:010BFB0000F9
:010BFC0000F8
:010BFD0000F7
:010BFE0000F6
:010BFF0000F5
:010C000000F3
:010C010000F2
:010C020000F1
:010C030000F0
:010C040000EF
:010C050000EE
:010C060000ED
:010C070000EC
:010C080000EB
:010C090000EA
:010C0A0000E9
:010C0B0000E8
:010C0C0000E7
:010C0D0000E6
:010C0E0000E5
:010C0F0000E4
:010C100000E3
:010C110000E2
:010C120000E1
:010C130000E0
:010C140000DF
:010C150000DE
:010C160000DD
:010C170000DC
:010C180000DB
:010C190000DA
:010C1A0000D9
:010C1B0000D8
:010C1C0000D7
:010C1D0000D6
:010C1E0000D5
:010C1F0000D4
:010C200000D3
:010C210000D2
:010C220000D1
:010C230000D0
:010C240000CF
:010C250000CE
:010C260000CD
:010C270000CC
:010C280000CB
:010C290000CA
:010C2A0000C9
:010C2B0000C8
:010C2C0000C7
:010C2D0000C6
:010C2E0000C5
:010C2F0000C4
:010C300000C3
:010C310000C2
:010C320000C1
:010C330000C0
:010C340000BF
:010C350000BE
:010C360000BD
:010C370000BC
:010C380000BB
:010C390000BA
:010C3A0000B9
:010C3B0000B8
:010C3C0000B7
:010C3D0000B6
:010C3E0000B5
:010C3F0000B4
:010C400000B3
:010C410000B2
:010C420000B1
:010C430000B0
:010C440000AF
:010C450000AE
:010C460000AD
:010C470000AC
:010C480000AB
:010C490000AA
:010C4A0000A9
:010C4B0000A8
:010C4C0000A7
:010C4D0000A6
:010C4E0000A5
:010C4F0000A4
:010C500000A3
:010C510000A2
:010C520000A1
:010C530000A0
:010C5400009F
:010C5500009E
:010C5600009D
:010C5700009C
:010C5800009B
:010C5900009A
:010C5A000099
:010C5B000098
:010C5C000097
:010C5D000096
:010C5E000095
:010C5F000094
:010C60000093
:010C61000092
:010C62000091
:010C63000090
:010C6400008F
:010C6500008E
:010C6600008D
:010C6700008C
:010C6800008B
:010C6900008A
:010C6A000089
:010C6B000088
:010C6C000087
:010C6D000086
:010C6E000085
:010C6F000084
:010C70000083
:010C71000082
:010C72000081
:010C73000080
:010C7400007F
:010C7500007E
:010C7600007D
:010C7700007C
:010C7800007B
:010C7900007A
:010C7A000079
:010C7B000078
:010C7C000077
:010C7D000076
:010C7E000075
:010C7F000074
:010C80000073
:010C81000072
:010C82000071
:010C83000070
:010C8400006F
:010C8500006E
:010C8600006D
:010C8700006C
:010C8800006B
:010C8900006A
:010C8A000069
:010C8B000068
:010C8C000067
:010C8D000066
:010C8E000065
:010C8F000064
:010C90000063
:010C91000062
:010C92000061
:010C93000060
:010C9400005F
:010C9500005E
:010C9600005D
:010C9700005C
:010C9800005B
:010C9900005A
:010C9A000059
:010C9B000058
:010C9C000057
:010C9D000056
:010C9E000055
:010C9F000054
:010CA0000053
:010CA1000052
:010CA2000051
:010CA3000050
:010CA400004F
:010CA500004E
:010CA600004D
:010CA700004C
:010CA800004B
:010CA900004A
:010CAA000049
:010CAB000048
:010CAC000047
:010CAD000046
:010CAE000045
:010CAF000044
:010CB0000043
:010CB1000042
:010CB2000041
:010CB3000040
:010CB400003F
:010CB500003E
:010CB600003D
:010CB700003C
:010CB800003B
:010CB900003A
:010CBA000039
:010CBB000038
:010CBC000037
:010CBD000036
:010CBE000035
:010CBF000034
:010CC0000033
:010CC1000032
:010CC2000031
:010CC3000030
:010CC400002F
:010CC500002E
:010CC600002D
:010CC700002C
:010CC800002B
:010CC900002A
:010CCA000029
:010CCB000028
:010CCC000027
:010CCD000026
:010CCE000025
:010CCF000024
:010CD0000023
:010CD1000022
:010CD2000021
:010CD3000020
:010CD400001F
:010CD500001E
:010CD600001D
:010CD700001C
:010CD800001B
:010CD900001A
:010CDA000019
:010CDB000018
:010CDC000017
:010CDD000016
:010CDE000015
:010CDF000014
:010CE0000013
:010CE1000012
:010CE2000011
:010CE3000010
:010CE400000F
:010CE500000E
:010CE600000D
:010CE700000C
:010CE800000B
:010CE900000A
:010CEA000009
:010CEB000008
:010CEC000007
:010CED000006
:010CEE000005
:010CEF000004
:010CF0000003
:010CF1000002
:010CF2000001
:010CF3000000
:010CF40000FF
:010CF50000FE
:010CF60000FD
:010CF70000FC
:010CF80000FB
:010CF90000FA
:010CFA0000F9
:010CFB0000F8
:010CFC0000F7
:010CFD0000F6
:010CFE0000F5
:010CFF0000F4
:010D000000F2
:010D010000F1
:010D020000F0
:010D030000EF
:010D040000EE
:010D050000ED
:010D060000EC
:010D070000EB
:010D080000EA
:010D090000E9
:010D0A0000E8
:010D0B0000E7
:010D0C0000E6
:010D0D0000E5
:010D0E0000E4
:010D0F0000E3
:010D100000E2
:010D110000E1
:010D120000E0
:010D130000DF
:010D140000DE
:010D150000DD
:010D160000DC
:010D170000DB
:010D180000DA
:010D190000D9
:010D1A0000D8
:010D1B0000D7
:010D1C0000D6
:010D1D0000D5
:010D1E0000D4
:010D1F0000D3
:010D200000D2
:010D210000D1
:010D220000D0
:010D230000CF
:010D240000CE
:010D250000CD
:010D260000CC
:010D270000CB
:010D280000CA
:010D290000C9
:010D2A0000C8
:010D2B0000C7
:010D2C0000C6
:010D2D0000C5
:010D2E0000C4
:010D2F0000C3
:010D300000C2
:010D310000C1
:010D320000C0
:010D330000BF
:010D340000BE
:010D350000BD
:010D360000BC
:010D370000BB
:010D380000BA
:010D390000B9
:010D3A0000B8
:010D3B0000B7
:010D3C0000B6
:010D3D0000B5
:010D3E0000B4
:010D3F0000B3
:010D400000B2
:010D410000B1
:010D420000B0
:010D430000AF
:010D440000AE
:010D450000AD
:010D460000AC
:010D470000AB
:010D480000AA
:010D490000A9
:010D4A0000A8
:010D4B0000A7
:010D4C0000A6
:010D4D0000A5
:010D4E0000A4
:010D4F0000A3
:010D500000A2
:010D510000A1
:010D520000A0
:010D5300009F
:010D5400009E
:010D5500009D
:010D5600009C
:010D5700009B
:010D5800009A
:010D59000099
:010D5A000098
:010D5B000097
:010D5C000096
:010D5D000095
:010D5E000094
:010D5F000093
:010D60000092
:010D61000091
:010D62000090
:010D6300008F
:010D6400008E
:010D6500008D
:010D6600008C
:010D6700008B
:010D6800008A
:010D69000089
:010D6A000088
:010D6B000087
:010D6C000086
:010D6D000085
:010D6E000084
:010D6F000083
:010D70000082
:010D71000081
:010D72000080
:010D7300007F
:010D7400007E
:010D7500007D
:010D7600007C
:010D7700007B
:010D7800007A
:010D79000079
:010D7A000078
:010D7B000077
:010D7C000076
:010D7D000075
:010D7E000074
:010D7F000073
:010D80000072
:010D81000071
:010D82000070
:010D8300006F
:010D8400006E
:010D8500006D
:010D8600006C
:010D8700006B
:010D8800006A
:010D89000069
:010D8A000068
:010D8B000067
:010D8C000066
:010D8D000065
:010D8E000064
:010D8F000063
:010D90000062
:010D91000061
:010D92000060
:010D9300005F
:010D9400005E
:010D9500005D
:010D9600005C
:010D9700005B
:010D9800005A
:010D99000059
:010D9A000058
:010D9B000057
:010D9C000056
:010D9D000055
:010D9E000054
:010D9F000053
:010DA0000052
:010DA1000051
:010DA2000050
:010DA300004F
:010DA400004E
:010DA500004D
:010DA600004C
:010DA700004B
:010DA800004A
:010DA9000049
:010DAA000048
:010DAB000047
:010DAC000046
:010DAD000045
:010DAE000044
:010DAF000043
:010DB0000042
:010DB1000041
:010DB2000040
:010DB300003F
:010DB400003E
:010DB500003D
:010DB600003C
:010DB700003B
:010DB800003A
:010DB9000039
:010DBA000038
:010DBB000037
:010DBC000036
:010DBD000035
:010DBE000034
:010DBF000033
:010DC0000032
:010DC1000031
:010DC2000030
:010DC300002F
:010DC400002E
:010DC500002D
:010DC600002C
:010DC700002B
:010DC800002A
:010DC9000029
:010DCA000028
:010DCB000027
:010DCC000026
:010DCD000025
:010DCE000024
:010DCF000023
:010DD0000022
:010DD1000021
:010DD2000020
:010DD300001F
:010DD400001E
:010DD500001D
:010DD600001C
:010DD700001B
:010DD800001A
:010DD9000019
:010DDA000018
:010DDB000017
:010DDC000016
:010DDD000015
:010DDE000014
:010DDF000013
:010DE0000012
:010DE1000011
:010DE2000010
:010DE300000F
:010DE400000E
:010DE500000D
:010DE600000C
:010DE700000B
:010DE800000A
:010DE9000009
:010DEA000008
:010DEB000007
:010DEC000006
:010DED000005
:010DEE000004
:010DEF000003
:010DF0000002
:010DF1000001
:010DF2000000
:010DF30000FF
:010DF40000FE
:010DF50000FD
:010DF60000FC
:010DF70000FB
:010DF80000FA
:010DF90000F9
:010DFA0000F8
:010DFB0000F7
:010DFC0000F6
:010DFD0000F5
:010DFE0000F4
:010DFF0000F3
:010E000000F1
:010E010000F0
:010E020000EF
:010E030000EE
:010E040000ED
:010E050000EC
:010E060000EB
:010E070000EA
:010E080000E9
:010E090000E8
:010E0A0000E7
:010E0B0000E6
:010E0C0000E5
:010E0D0000E4
:010E0E0000E3
:010E0F0000E2
:010E100000E1
:010E110000E0
:010E120000DF
:010E130000DE
:010E140000DD
:010E150000DC
:010E160000DB
:010E170000DA
:010E180000D9
:010E190000D8
:010E1A0000D7
:010E1B0000D6
:010E1C0000D5
:010E1D0000D4
:010E1E0000D3
:010E1F0000D2
:010E200000D1
:010E210000D0
:010E220000CF
:010E230000CE
:010E240000CD
:010E250000CC
:010E260000CB
:010E270000CA
:010E280000C9
:010E290000C8
:010E2A0000C7
:010E2B0000C6
:010E2C0000C5
:010E2D0000C4
:010E2E0000C3
:010E2F0000C2
:010E300000C1
:010E310000C0
:010E320000BF
:010E330000BE
:010E340000BD
:010E350000BC
:010E360000BB
:010E370000BA
:010E380000B9
:010E390000B8
:010E3A0000B7
:010E3B0000B6
:010E3C0000B5
:010E3D0000B4
:010E3E0000B3
:010E3F0000B2
:010E400000B1
:010E410000B0
:010E420000AF
:010E430000AE
:010E440000AD
:010E450000AC
:010E460000AB
:010E470000AA
:010E480000A9
:010E490000A8
:010E4A0000A7
:010E4B0000A6
:010E4C0000A5
:010E4D0000A4
:010E4E0000A3
:010E4F0000A2
:010E500000A1
:010E510000A0
:010E5200009F
:010E5300009E
:010E5400009D
:010E5500009C
:010E5600009B
:010E5700009A
:010E58000099
:010E59000098
:010E5A000097
:010E5B000096
:010E5C000095
:010E5D000094
:010E5E000093
:010E5F000092
:010E60000091
:010E61000090
:010E6200008F
:010E6300008E
:010E6400008D
:010E6500008C
:010E6600008B
:010E6700008A
:010E68000089
:010E69000088
:010E6A000087
:010E6B000086
:010E6C000085
:010E6D000084
:010E6E000083
:010E6F000082
:010E70000081
:010E71000080
:010E7200007F
:010E7300007E
:010E7400007D
:010E7500007C
:010E7600007B
:010E7700007A
:010E78000079
:010E79000078
:010E7A000077
:010E7B000076
:010E7C000075
:010E7D000074
:010E7E000073
:010E7F000072
:010E80000071
:010E81000070
:010E8200006F
:010E8300006E
:010E8400006D
:010E8500006C
:010E8600006B
:010E8700006A
:010E88000069
:010E89000068
:010E8A000067
:010E8B000066
:010E8C000065
:010E8D000064
:010E8E000063
:010E8F000062
:010E90000061
:010E91000060
:010E9200005F
:010E9300005E
:010E9400005D
:010E9500005C
:010E9600005B
:010E9700005A
:010E98000059
:010E99000058
:010E9A000057
:010E9B000056
:010E9C000055
:010E9D000054
:010E9E000053
:010E9F000052
:010EA0000051
:010EA1000050
:010EA200004F
:010EA300004E
:010EA400004D
:010EA500004C
:010EA600004B
:010EA700004A
:010EA8000049
:010EA9000048
:010EAA000047
:010EAB000046
:010EAC000045
:010EAD000044
:010EAE000043
:010EAF000042
:010EB0000041
:010EB1000040
:010EB200003F
:010EB300003E
:010EB400003D
:010EB500003C
:010EB600003B
:010EB700003A
:010EB8000039
:010EB9000038
:010EBA000037
:010EBB000036
:010EBC000035
:010EBD000034
:010EBE000033
:010EBF000032
:010EC0000031
:010EC1000030
:010EC200002F
:010EC300002E
:010EC400002D
:010EC500002C
:010EC600002B
:010EC700002A
:010EC8000029
:010EC9000028
:010ECA000027
:010ECB000026
:010ECC000025
:010ECD000024
:010ECE000023
:010ECF000022
:010ED0000021
:010ED1000020
:010ED200001F
:010ED300001E
:010ED400001D
:010ED500001C
:010ED600001B
:010ED700001A
:010ED8000019
:010ED9000018
:010EDA000017
:010EDB000016
:010EDC000015
:010EDD000014
:010EDE000013
:010EDF000012
:010EE0000011
:010EE1000010
:010EE200000F
:010EE300000E
:010EE400000D
:010EE500000C
:010EE600000B
:010EE700000A
:010EE8000009
:010EE9000008
:010EEA000007
:010EEB000006
:010EEC000005
:010EED000004
:010EEE000003
:010EEF000002
:010EF0000001
:010EF1000000
:010EF20000FF
:010EF30000FE
:010EF40000FD
:010EF50000FC
:010EF60000FB
:010EF70000FA
:010EF80000F9
:010EF90000F8
:010EFA0000F7
:010EFB0000F6
:010EFC0000F5
:010EFD0000F4
:010EFE0000F3
:010EFF0000F2
:010F000000F0
:010F010000EF
:010F020000EE
:010F030000ED
:010F040000EC
:010F050000EB
:010F060000EA
:010F070000E9
:010F080000E8
:010F090000E7
:010F0A0000E6
:010F0B0000E5
:010F0C0000E4
:010F0D0000E3
:010F0E0000E2
:010F0F0000E1
:010F100000E0
:010F110000DF
:010F120000DE
:010F130000DD
:010F140000DC
:010F150000DB
:010F160000DA
:010F170000D9
:010F180000D8
:010F190000D7
:010F1A0000D6
:010F1B0000D5
:010F1C0000D4
:010F1D0000D3
:010F1E0000D2
:010F1F0000D1
:010F200000D0
:010F210000CF
:010F220000CE
:010F230000CD
:010F240000CC
:010F250000CB
:010F260000CA
:010F270000C9
:010F280000C8
:010F290000C7
:010F2A0000C6
:010F2B0000C5
:010F2C0000C4
:010F2D0000C3
:010F2E0000C2
:010F2F0000C1
:010F300000C0
:010F310000BF
:010F320000BE
:010F330000BD
:010F340000BC
:010F350000BB
:010F360000BA
:010F370000B9
:010F380000B8
:010F390000B7
:010F3A0000B6
:010F3B0000B5
:010F3C0000B4
:010F3D0000B3
:010F3E0000B2
:010F3F0000B1
:010F400000B0
:010F410000AF
:010F420000AE
:010F430000AD
:010F440000AC
:010F450000AB
:010F460000AA
:010F470000A9
:010F480000A8
:010F490000A7
:010F4A0000A6
:010F4B0000A5
:010F4C0000A4
:010F4D0000A3
:010F4E0000A2
:010F4F0000A1
:010F500000A0
:010F5100009F
:010F5200009E
:010F5300009D
:010F5400009C
:010F5500009B
:010F5600009A
:010F57000099
:010F58000098
:010F59000097
:010F5A000096
:010F5B000095
:010F5C000094
:010F5D000093
:010F5E000092
:010F5F000091
:010F60000090
:010F6100008F
:010F6200008E
:010F6300008D
:010F6400008C
:010F6500008B
:010F6600008A
:010F67000089
:010F68000088
:010F69000087
:010F6A000086
:010F6B000085
:010F6C000084
:010F6D000083
:010F6E000082
:010F6F000081
:010F70000080
:010F7100007F
:010F7200007E
:010F7300007D
:010F7400007C
:010F7500007B
:010F7600007A
:010F77000079
:010F78000078
:010F79000077
:010F7A000076
:010F7B000075
:010F7C000074
:010F7D000073
:010F7E000072
:010F7F000071
:010F80000070
:010F8100006F
:010F8200006E
:010F8300006D
:010F8400006C
:010F8500006B
:010F8600006A
:010F87000069
:010F88000068
:010F89000067
:010F8A000066
:010F8B000065
:010F8C000064
:010F8D000063
:010F8E000062
:010F8F000061
:010F90000060
:010F9100005F
:010F9200005E
:010F9300005D
:010F9400005C
:010F9500005B
:010F9600005A
:010F97000059
:010F98000058
:010F99000057
:010F9A000056
:010F9B000055
:010F9C000054
:010F9D000053
:010F9E000052
:010F9F000051
:010FA0000050
:010FA100004F
:010FA200004E
:010FA300004D
:010FA400004C
:010FA500004B
:010FA600004A
:010FA7000049
:010FA8000048
:010FA9000047
:010FAA000046
:010FAB000045
:010FAC000044
:010FAD000043
:010FAE000042
:010FAF000041
:010FB0000040
:010FB100003F
:010FB200003E
:010FB300003D
:010FB400003C
:010FB500003B
:010FB600003A
:010FB7000039
:010FB8000038
:010FB9000037
:010FBA000036
:010FBB000035
:010FBC000034
:010FBD000033
:010FBE000032
:010FBF000031
:010FC0000030
:010FC100002F
:010FC200002E
:010FC300002D
:010FC400002C
:010FC500002B
:010FC600002A
:010FC7000029
:010FC8000028
:010FC9000027
:010FCA000026
:010FCB000025
:010FCC000024
:010FCD000023
:010FCE000022
:010FCF000021
:010FD0000020
:010FD100001F
:010FD200001E
:010FD300001D
:010FD400001C
:010FD500001B
:010FD600001A
:010FD7000019
:010FD8000018
:010FD9000017
:010FDA000016
:010FDB000015
:010FDC000014
:010FDD000013
:010FDE000012
:010FDF000011
:010FE0000010
:010FE100000F
:010FE200000E
:010FE300000D
:010FE400000C
:010FE500000B
:010FE600000A
:010FE7000009
:010FE8000008
:010FE9000007
:010FEA000006
:010FEB000005
:010FEC000004
:010FED000003
:010FEE000002
:010FEF000001
:010FF0000000
:010FF10000FF
:010FF20000FE
:010FF30000FD
:010FF40000FC
:010FF50000FB
:010FF60000FA
:010FF70000F9
:010FF80000F8
:010FF90000F7
:010FFA0000F6
:010FFB0000F5
:010FFC0000F4
:010FFD0000F3
:010FFE0000F2
:010FFF0000F1
:0110000000EF
:0110010000EE
:0110020000ED
:0110030000EC
:0110040000EB
:0110050000EA
:0110060000E9
:0110070000E8
:0110080000E7
:0110090000E6
:01100A0000E5
:01100B0000E4
:01100C0000E3
:01100D0000E2
:01100E0000E1
:01100F0000E0
:0110100000DF
:0110110000DE
:0110120000DD
:0110130000DC
:0110140000DB
:0110150000DA
:0110160000D9
:0110170000D8
:0110180000D7
:0110190000D6
:01101A0000D5
:01101B0000D4
:01101C0000D3
:01101D0000D2
:01101E0000D1
:01101F0000D0
:0110200000CF
:0110210000CE
:0110220000CD
:0110230000CC
:0110240000CB
:0110250000CA
:0110260000C9
:0110270000C8
:0110280000C7
:0110290000C6
:01102A0000C5
:01102B0000C4
:01102C0000C3
:01102D0000C2
:01102E0000C1
:01102F0000C0
:0110300000BF
:0110310000BE
:0110320000BD
:0110330000BC
:0110340000BB
:0110350000BA
:0110360000B9
:0110370000B8
:0110380000B7
:0110390000B6
:01103A0000B5
:01103B0000B4
:01103C0000B3
:01103D0000B2
:01103E0000B1
:01103F0000B0
:0110400000AF
:0110410000AE
:0110420000AD
:0110430000AC
:0110440000AB
:0110450000AA
:0110460000A9
:0110470000A8
:0110480000A7
:0110490000A6
:01104A0000A5
:01104B0000A4
:01104C0000A3
:01104D0000A2
:01104E0000A1
:01104F0000A0
:01105000009F
:01105100009E
:01105200009D
:01105300009C
:01105400009B
:01105500009A
:011056000099
:011057000098
:011058000097
:011059000096
:01105A000095
:01105B000094
:01105C000093
:01105D000092
:01105E000091
:01105F000090
:01106000008F
:01106100008E
:01106200008D
:01106300008C
:01106400008B
:01106500008A
:011066000089
:011067000088
:011068000087
:011069000086
:01106A000085
:01106B000084
:01106C000083
:01106D000082
:01106E000081
:01106F000080
:01107000007F
:01107100007E
:01107200007D
:01107300007C
:01107400007B
:01107500007A
:011076000079
:011077000078
:011078000077
:011079000076
:01107A000075
:01107B000074
:01107C000073
:01107D000072
:01107E000071
:01107F000070
:01108000006F
:01108100006E
:01108200006D
:01108300006C
:01108400006B
:01108500006A
:011086000069
:011087000068
:011088000067
:011089000066
:01108A000065
:01108B000064
:01108C000063
:01108D000062
:01108E000061
:01108F000060
:01109000005F
:01109100005E
:01109200005D
:01109300005C
:01109400005B
:01109500005A
:011096000059
:011097000058
:011098000057
:011099000056
:01109A000055
:01109B000054
:01109C000053
:01109D000052
:01109E000051
:01109F000050
:0110A000004F
:0110A100004E
:0110A200004D
:0110A300004C
:0110A400004B
:0110A500004A
:0110A6000049
:0110A7000048
:0110A8000047
:0110A9000046
:0110AA000045
:0110AB000044
:0110AC000043
:0110AD000042
:0110AE000041
:0110AF000040
:0110B000003F
:0110B100003E
:0110B200003D
:0110B300003C
:0110B400003B
:0110B500003A
:0110B6000039
:0110B7000038
:0110B8000037
:0110B9000036
:0110BA000035
:0110BB000034
:0110BC000033
:0110BD000032
:0110BE000031
:0110BF000030
:0110C000002F
:0110C100002E
:0110C200002D
:0110C300002C
:0110C400002B
:0110C500002A
:0110C6000029
:0110C7000028
:0110C8000027
:0110C9000026
:0110CA000025
:0110CB000024
:0110CC000023
:0110CD000022
:0110CE000021
:0110CF000020
:0110D000001F
:0110D100001E
:0110D200001D
:0110D300001C
:0110D400001B
:0110D500001A
:0110D6000019
:0110D7000018
:0110D8000017
:0110D9000016
:0110DA000015
:0110DB000014
:0110DC000013
:0110DD000012
:0110DE000011
:0110DF000010
:0110E000000F
:0110E100000E
:0110E200000D
:0110E300000C
:0110E400000B
:0110E500000A
:0110E6000009
:0110E7000008
:0110E8000007
:0110E9000006
:0110EA000005
:0110EB000004
:0110EC000003
:0110ED000002
:0110EE000001
:0110EF000000
:0110F00000FF
:0110F10000FE
:0110F20000FD
:0110F30000FC
:0110F40000FB
:0110F50000FA
:0110F60000F9
:0110F70000F8
:0110F80000F7
:0110F90000F6
:0110FA0000F5
:0110FB0000F4
:0110FC0000F3
:0110FD0000F2
:0110FE0000F1
:0110FF0000F0
:0111000000EE
:0111010000ED
:0111020000EC
:0111030000EB
:0111040000EA
:0111050000E9
:0111060000E8
:0111070000E7
:0111080000E6
:0111090000E5
:01110A0000E4
:01110B0000E3
:01110C0000E2
:01110D0000E1
:01110E0000E0
:01110F0000DF
:0111100000DE
:0111110000DD
:0111120000DC
:0111130000DB
:0111140000DA
:0111150000D9
:0111160000D8
:0111170000D7
:0111180000D6
:0111190000D5
:01111A0000D4
:01111B0000D3
:01111C0000D2
:01111D0000D1
:01111E0000D0
:01111F0000CF
:0111200000CE
:0111210000CD
:0111220000CC
:0111230000CB
:0111240000CA
:0111250000C9
:0111260000C8
:0111270000C7
:0111280000C6
:0111290000C5
:01112A0000C4
:01112B0000C3
:01112C0000C2
:01112D0000C1
:01112E0000C0
:01112F0000BF
:0111300000BE
:0111310000BD
:0111320000BC
:0111330000BB
:0111340000BA
:0111350000B9
:0111360000B8
:0111370000B7
:0111380000B6
:0111390000B5
:01113A0000B4
:01113B0000B3
:01113C0000B2
:01113D0000B1
:01113E0000B0
:01113F0000AF
:0111400000AE
:0111410000AD
:0111420000AC
:0111430000AB
:0111440000AA
:0111450000A9
:0111460000A8
:0111470000A7
:0111480000A6
:0111490000A5
:01114A0000A4
:01114B0000A3
:01114C0000A2
:01114D0000A1
:01114E0000A0
:01114F00009F
:01115000009E
:01115100009D
:01115200009C
:01115300009B
:01115400009A
:011155000099
:011156000098
:011157000097
:011158000096
:011159000095
:01115A000094
:01115B000093
:01115C000092
:01115D000091
:01115E000090
:01115F00008F
:01116000008E
:01116100008D
:01116200008C
:01116300008B
:01116400008A
:011165000089
:011166000088
:011167000087
:011168000086
:011169000085
:01116A000084
:01116B000083
:01116C000082
:01116D000081
:01116E000080
:01116F00007F
:01117000007E
:01117100007D
:01117200007C
:01117300007B
:01117400007A
:011175000079
:011176000078
:011177000077
:011178000076
:011179000075
:01117A000074
:01117B000073
:01117C000072
:01117D000071
:01117E000070
:01117F00006F
:01118000006E
:01118100006D
:01118200006C
:01118300006B
:01118400006A
:011185000069
:011186000068
:011187000067
:011188000066
:011189000065
:01118A000064
:01118B000063
:01118C000062
:01118D000061
:01118E000060
:01118F00005F
:01119000005E
:01119100005D
:01119200005C
:01119300005B
:01119400005A
:011195000059
:011196000058
:011197000057
:011198000056
:011199000055
:01119A000054
:01119B000053
:01119C000052
:01119D000051
:01119E000050
:01119F00004F
:0111A000004E
:0111A100004D
:0111A200004C
:0111A300004B
:0111A400004A
:0111A5000049
:0111A6000048
:0111A7000047
:0111A8000046
:0111A9000045
:0111AA000044
:0111AB000043
:0111AC000042
:0111AD000041
:0111AE000040
:0111AF00003F
:0111B000003E
:0111B100003D
:0111B200003C
:0111B300003B
:0111B400003A
:0111B5000039
:0111B6000038
:0111B7000037
:0111B8000036
:0111B9000035
:0111BA000034
:0111BB000033
:0111BC000032
:0111BD000031
:0111BE000030
:0111BF00002F
:0111C000002E
:0111C100002D
:0111C200002C
:0111C300002B
:0111C400002A
:0111C5000029
:0111C6000028
:0111C7000027
:0111C8000026
:0111C9000025
:0111CA000024
:0111CB000023
:0111CC000022
:0111CD000021
:0111CE000020
:0111CF00001F
:0111D000001E
:0111D100001D
:0111D200001C
:0111D300001B
:0111D400001A
:0111D5000019
:0111D6000018
:0111D7000017
:0111D8000016
:0111D9000015
:0111DA000014
:0111DB000013
:0111DC000012
:0111DD000011
:0111DE000010
:0111DF00000F
:0111E000000E
:0111E100000D
:0111E200000C
:0111E300000B
:0111E400000A
:0111E5000009
:0111E6000008
:0111E7000007
:0111E8000006
:0111E9000005
:0111EA000004
:0111EB000003
:0111EC000002
:0111ED000001
:0111EE000000
:0111EF0000FF
:0111F00000FE
:0111F10000FD
:0111F20000FC
:0111F30000FB
:0111F40000FA
:0111F50000F9
:0111F60000F8
:0111F70000F7
:0111F80000F6
:0111F90000F5
:0111FA0000F4
:0111FB0000F3
:0111FC0000F2
:0111FD0000F1
:0111FE0000F0
:0111FF0000EF
:0112000000ED
:0112010000EC
:0112020000EB
:0112030000EA
:0112040000E9
:0112050000E8
:0112060000E7
:0112070000E6
:0112080000E5
:0112090000E4
:01120A0000E3
:01120B0000E2
:01120C0000E1
:01120D0000E0
:01120E0000DF
:01120F0000DE
:0112100000DD
:0112110000DC
:0112120000DB
:0112130000DA
:0112140000D9
:0112150000D8
:0112160000D7
:0112170000D6
:0112180000D5
:0112190000D4
:01121A0000D3
:01121B0000D2
:01121C0000D1
:01121D0000D0
:01121E0000CF
:01121F0000CE
:0112200000CD
:0112210000CC
:0112220000CB
:0112230000CA
:0112240000C9
:0112250000C8
:0112260000C7
:0112270000C6
:0112280000C5
:0112290000C4
:01122A0000C3
:01122B0000C2
:01122C0000C1
:01122D0000C0
:01122E0000BF
:01122F0000BE
:0112300000BD
:0112310000BC
:0112320000BB
:0112330000BA
:0112340000B9
:0112350000B8
:0112360000B7
:0112370000B6
:0112380000B5
:0112390000B4
:01123A0000B3
:01123B0000B2
:01123C0000B1
:01123D0000B0
:01123E0000AF
:01123F0000AE
:0112400000AD
:0112410000AC
:0112420000AB
:0112430000AA
:0112440000A9
:0112450000A8
:0112460000A7
:0112470000A6
:0112480000A5
:0112490000A4
:01124A0000A3
:01124B0000A2
:01124C0000A1
:01124D0000A0
:01124E00009F
:01124F00009E
:01125000009D
:01125100009C
:01125200009B
:01125300009A
:011254000099
:011255000098
:011256000097
:011257000096
:011258000095
:011259000094
:01125A000093
:01125B000092
:01125C000091
:01125D000090
:01125E00008F
:01125F00008E
:01126000008D
:01126100008C
:01126200008B
:01126300008A
:011264000089
:011265000088
:011266000087
:011267000086
:011268000085
:011269000084
:01126A000083
:01126B000082
:01126C000081
:01126D000080
:01126E00007F
:01126F00007E
:01127000007D
:01127100007C
:01127200007B
:01127300007A
:011274000079
:011275000078
:011276000077
:011277000076
:011278000075
:011279000074
:01127A000073
:01127B000072
:01127C000071
:01127D000070
:01127E00006F
:01127F00006E
:01128000006D
:01128100006C
:01128200006B
:01128300006A
:011284000069
:011285000068
:011286000067
:011287000066
:011288000065
:011289000064
:01128A000063
:01128B000062
:01128C000061
:01128D000060
:01128E00005F
:01128F00005E
:01129000005D
:01129100005C
:01129200005B
:01129300005A
:011294000059
:011295000058
:011296000057
:011297000056
:011298000055
:011299000054
:01129A000053
:01129B000052
:01129C000051
:01129D000050
:01129E00004F
:01129F00004E
:0112A000004D
:0112A100004C
:0112A200004B
:0112A300004A
:0112A4000049
:0112A5000048
:0112A6000047
:0112A7000046
:0112A8000045
:0112A9000044
:0112AA000043
:0112AB000042
:0112AC000041
:0112AD000040
:0112AE00003F
:0112AF00003E
:0112B000003D
:0112B100003C
:0112B200003B
:0112B300003A
:0112B4000039
:0112B5000038
:0112B6000037
:0112B7000036
:0112B8000035
:0112B9000034
:0112BA000033
:0112BB000032
:0112BC000031
:0112BD000030
:0112BE00002F
:0112BF00002E
:0112C000002D
:0112C100002C
:0112C200002B
:0112C300002A
:0112C4000029
:0112C5000028
:0112C6000027
:0112C7000026
:0112C8000025
:0112C9000024
:0112CA000023
:0112CB000022
:0112CC000021
:0112CD000020
:0112CE00001F
:0112CF00001E
:0112D000001D
:0112D100001C
:0112D200001B
:0112D300001A
:0112D4000019
:0112D5000018
:0112D6000017
:0112D7000016
:0112D8000015
:0112D9000014
:0112DA000013
:0112DB000012
:0112DC000011
:0112DD000010
:0112DE00000F
:0112DF00000E
:0112E000000D
:0112E100000C
:0112E200000B
:0112E300000A
:0112E4000009
:0112E5000008
:0112E6000007
:0112E7000006
:0112E8000005
:0112E9000004
:0112EA000003
:0112EB000002
:0112EC000001
:0112ED000000
:0112EE0000FF
:0112EF0000FE
:0112F00000FD
:0112F10000FC
:0112F20000FB
:0112F30000FA
:0112F40000F9
:0112F50000F8
:0112F60000F7
:0112F70000F6
:0112F80000F5
:0112F90000F4
:0112FA0000F3
:0112FB0000F2
:0112FC0000F1
:0112FD0000F0
:0112FE0000EF
:0112FF0000EE
:0113000000EC
:0113010000EB
:0113020000EA
:0113030000E9
:0113040000E8
:0113050000E7
:0113060000E6
:0113070000E5
:0113080000E4
:0113090000E3
:01130A0000E2
:01130B0000E1
:01130C0000E0
:01130D0000DF
:01130E0000DE
:01130F0000DD
:0113100000DC
:0113110000DB
:0113120000DA
:0113130000D9
:0113140000D8
:0113150000D7
:0113160000D6
:0113170000D5
:0113180000D4
:0113190000D3
:01131A0000D2
:01131B0000D1
:01131C0000D0
:01131D0000CF
:01131E0000CE
:01131F0000CD
:0113200000CC
:0113210000CB
:0113220000CA
:0113230000C9
:0113240000C8
:0113250000C7
:0113260000C6
:0113270000C5
:0113280000C4
:0113290000C3
:01132A0000C2
:01132B0000C1
:01132C0000C0
:01132D0000BF
:01132E0000BE
:01132F0000BD
:0113300000BC
:0113310000BB
:0113320000BA
:0113330000B9
:0113340000B8
:0113350000B7
:0113360000B6
:0113370000B5
:0113380000B4
:0113390000B3
:01133A0000B2
:01133B0000B1
:01133C0000B0
:01133D0000AF
:01133E0000AE
:01133F0000AD
:0113400000AC
:0113410000AB
:0113420000AA
:0113430000A9
:0113440000A8
:0113450000A7
:0113460000A6
:0113470000A5
:0113480000A4
:0113490000A3
:01134A0000A2
:01134B0000A1
:01134C0000A0
:01134D00009F
:01134E00009E
:01134F00009D
:01135000009C
:01135100009B
:01135200009A
:011353000099
:011354000098
:011355000097
:011356000096
:011357000095
:011358000094
:011359000093
:01135A000092
:01135B000091
:01135C000090
:01135D00008F
:01135E00008E
:01135F00008D
:01136000008C
:01136100008B
:01136200008A
:011363000089
:011364000088
:011365000087
:011366000086
:011367000085
:011368000084
:011369000083
:01136A000082
:01136B000081
:01136C000080
:01136D00007F
:01136E00007E
:01136F00007D
:01137000007C
:01137100007B
:01137200007A
:011373000079
:011374000078
:011375000077
:011376000076
:011377000075
:011378000074
:011379000073
:01137A000072
:01137B000071
:01137C000070
:01137D00006F
:01137E00006E
:01137F00006D
:01138000006C
:01138100006B
:01138200006A
:011383000069
:011384000068
:011385000067
:011386000066
:011387000065
:011388000064
:011389000063
:01138A000062
:01138B000061
:01138C000060
:01138D00005F
:01138E00005E
:01138F00005D
:01139000005C
:01139100005B
:01139200005A
:011393000059
:011394000058
:011395000057
:011396000056
:011397000055
:011398000054
:011399000053
:01139A000052
:01139B000051
:01139C000050
:01139D00004F
:01139E00004E
:01139F00004D
:0113A000004C
:0113A100004B
:0113A200004A
:0113A3000049
:0113A4000048
:0113A5000047
:0113A6000046
:0113A7000045
:0113A8000044
:0113A9000043
:0113AA000042
:0113AB000041
:0113AC000040
:0113AD00003F
:0113AE00003E
:0113AF00003D
:0113B000003C
:0113B100003B
:0113B200003A
:0113B3000039
:0113B4000038
:0113B5000037
:0113B6000036
:0113B7000035
:0113B8000034
:0113B9000033
:0113BA000032
:0113BB000031
:0113BC000030
:0113BD00002F
:0113BE00002E
:0113BF00002D
:0113C000002C
:0113C100002B
:0113C200002A
:0113C3000029
:0113C4000028
:0113C5000027
:0113C6000026
:0113C7000025
:0113C8000024
:0113C9000023
:0113CA000022
:0113CB000021
:0113CC000020
:0113CD00001F
:0113CE00001E
:0113CF00001D
:0113D000001C
:0113D100001B
:0113D200001A
:0113D3000019
:0113D4000018
:0113D5000017
:0113D6000016
:0113D7000015
:0113D8000014
:0113D9000013
:0113DA000012
:0113DB000011
:0113DC000010
:0113DD00000F
:0113DE00000E
:0113DF00000D
:0113E000000C
:0113E100000B
:0113E200000A
:0113E3000009
:0113E4000008
:0113E5000007
:0113E6000006
:0113E7000005
:0113E8000004
:0113E9000003
:0113EA000002
:0113EB000001
:0113EC000000
:0113ED0000FF
:0113EE0000FE
:0113EF0000FD
:0113F00000FC
:0113F10000FB
:0113F20000FA
:0113F30000F9
:0113F40000F8
:0113F50000F7
:0113F60000F6
:0113F70000F5
:0113F80000F4
:0113F90000F3
:0113FA0000F2
:0113FB0000F1
:0113FC0000F0
:0113FD0000EF
:0113FE0000EE
:0113FF0000ED
:0114000000EB
:0114010000EA
:0114020000E9
:0114030000E8
:0114040000E7
:0114050000E6
:0114060000E5
:0114070000E4
:0114080000E3
:0114090000E2
:01140A0000E1
:01140B0000E0
:01140C0000DF
:01140D0000DE
:01140E0000DD
:01140F0000DC
:0114100000DB
:0114110000DA
:0114120000D9
:0114130000D8
:0114140000D7
:0114150000D6
:0114160000D5
:0114170000D4
:0114180000D3
:0114190000D2
:01141A0000D1
:01141B0000D0
:01141C0000CF
:01141D0000CE
:01141E0000CD
:01141F0000CC
:0114200000CB
:0114210000CA
:0114220000C9
:0114230000C8
:0114240000C7
:0114250000C6
:0114260000C5
:0114270000C4
:0114280000C3
:0114290000C2
:01142A0000C1
:01142B0000C0
:01142C0000BF
:01142D0000BE
:01142E0000BD
:01142F0000BC
:0114300000BB
:0114310000BA
:0114320000B9
:0114330000B8
:0114340000B7
:0114350000B6
:0114360000B5
:0114370000B4
:0114380000B3
:0114390000B2
:01143A0000B1
:01143B0000B0
:01143C0000AF
:01143D0000AE
:01143E0000AD
:01143F0000AC
:0114400000AB
:0114410000AA
:0114420000A9
:0114430000A8
:0114440000A7
:0114450000A6
:0114460000A5
:0114470000A4
:0114480000A3
:0114490000A2
:01144A0000A1
:01144B0000A0
:01144C00009F
:01144D00009E
:01144E00009D
:01144F00009C
:01145000009B
:01145100009A
:011452000099
:011453000098
:011454000097
:011455000096
:011456000095
:011457000094
:011458000093
:011459000092
:01145A000091
:01145B000090
:01145C00008F
:01145D00008E
:01145E00008D
:01145F00008C
:01146000008B
:01146100008A
:011462000089
:011463000088
:011464000087
:011465000086
:011466000085
:011467000084
:011468000083
:011469000082
:01146A000081
:01146B000080
:01146C00007F
:01146D00007E
:01146E00007D
:01146F00007C
:01147000007B
:01147100007A
:011472000079
:011473000078
:011474000077
:011475000076
:011476000075
:011477000074
:011478000073
:011479000072
:01147A000071
:01147B000070
:01147C00006F
:01147D00006E
:01147E00006D
:01147F00006C
:01148000006B
:01148100006A
:011482000069
:011483000068
:011484000067
:011485000066
:011486000065
:011487000064
:011488000063
:011489000062
:01148A000061
:01148B000060
:01148C00005F
:01148D00005E
:01148E00005D
:01148F00005C
:01149000005B
:01149100005A
:011492000059
:011493000058
:011494000057
:011495000056
:011496000055
:011497000054
:011498000053
:011499000052
:01149A000051
:01149B000050
:01149C00004F
:01149D00004E
:01149E00004D
:01149F00004C
:0114A000004B
:0114A100004A
:0114A2000049
:0114A3000048
:0114A4000047
:0114A5000046
:0114A6000045
:0114A7000044
:0114A8000043
:0114A9000042
:0114AA000041
:0114AB000040
:0114AC00003F
:0114AD00003E
:0114AE00003D
:0114AF00003C
:0114B000003B
:0114B100003A
:0114B2000039
:0114B3000038
:0114B4000037
:0114B5000036
:0114B6000035
:0114B7000034
:0114B8000033
:0114B9000032
:0114BA000031
:0114BB000030
:0114BC00002F
:0114BD00002E
:0114BE00002D
:0114BF00002C
:0114C000002B
:0114C100002A
:0114C2000029
:0114C3000028
:0114C4000027
:0114C5000026
:0114C6000025
:0114C7000024
:0114C8000023
:0114C9000022
:0114CA000021
:0114CB000020
:0114CC00001F
:0114CD00001E
:0114CE00001D
:0114CF00001C
:0114D000001B
:0114D100001A
:0114D2000019
:0114D3000018
:0114D4000017
:0114D5000016
:0114D6000015
:0114D7000014
:0114D8000013
:0114D9000012
:0114DA000011
:0114DB000010
:0114DC00000F
:0114DD00000E
:0114DE00000D
:0114DF00000C
:0114E000000B
:0114E100000A
:0114E2000009
:0114E3000008
:0114E4000007
:0114E5000006
:0114E6000005
:0114E7000004
:0114E8000003
:0114E9000002
:0114EA000001
:0114EB000000
:0114EC0000FF
:0114ED0000FE
:0114EE0000FD
:0114EF0000FC
:0114F00000FB
:0114F10000FA
:0114F20000F9
:0114F30000F8
:0114F40000F7
:0114F50000F6
:0114F60000F5
:0114F70000F4
:0114F80000F3
:0114F90000F2
:0114FA0000F1
:0114FB0000F0
:0114FC0000EF
:0114FD0000EE
:0114FE0000ED
:0114FF0000EC
:0115000000EA
:0115010000E9
:0115020000E8
:0115030000E7
:0115040000E6
:0115050000E5
:0115060000E4
:0115070000E3
:0115080000E2
:0115090000E1
:01150A0000E0
:01150B0000DF
:01150C0000DE
:01150D0000DD
:01150E0000DC
:01150F0000DB
:0115100000DA
:0115110000D9
:0115120000D8
:0115130000D7
:0115140000D6
:0115150000D5
:0115160000D4
:0115170000D3
:0115180000D2
:0115190000D1
:01151A0000D0
:01151B0000CF
:01151C0000CE
:01151D0000CD
:01151E0000CC
:01151F0000CB
:0115200000CA
:0115210000C9
:0115220000C8
:0115230000C7
:0115240000C6
:0115250000C5
:0115260000C4
:0115270000C3
:0115280000C2
:0115290000C1
:01152A0000C0
:01152B0000BF
:01152C0000BE
:01152D0000BD
:01152E0000BC
:01152F0000BB
:0115300000BA
:0115310000B9
:0115320000B8
:0115330000B7
:0115340000B6
:0115350000B5
:0115360000B4
:0115370000B3
:0115380000B2
:0115390000B1
:01153A0000B0
:01153B0000AF
:01153C0000AE
:01153D0000AD
:01153E0000AC
:01153F0000AB
:0115400000AA
:0115410000A9
:0115420000A8
:0115430000A7
:0115440000A6
:0115450000A5
:0115460000A4
:0115470000A3
:0115480000A2
:0115490000A1
:01154A0000A0
:01154B00009F
:01154C00009E
:01154D00009D
:01154E00009C
:01154F00009B
:01155000009A
:011551000099
:011552000098
:011553000097
:011554000096
:011555000095
:011556000094
:011557000093
:011558000092
:011559000091
:01155A000090
:01155B00008F
:01155C00008E
:01155D00008D
:01155E00008C
:01155F00008B
:01156000008A
:011561000089
:011562000088
:011563000087
:011564000086
:011565000085
:011566000084
:011567000083
:011568000082
:011569000081
:01156A000080
:01156B00007F
:01156C00007E
:01156D00007D
:01156E00007C
:01156F00007B
:01157000007A
:011571000079
:011572000078
:011573000077
:011574000076
:011575000075
:011576000074
:011577000073
:011578000072
:011579000071
:01157A000070
:01157B00006F
:01157C00006E
:01157D00006D
:01157E00006C
:01157F00006B
:01158000006A
:011581000069
:011582000068
:011583000067
:011584000066
:011585000065
:011586000064
:011587000063
:011588000062
:011589000061
:01158A000060
:01158B00005F
:01158C00005E
:01158D00005D
:01158E00005C
:01158F00005B
:01159000005A
:011591000059
:011592000058
:011593000057
:011594000056
:011595000055
:011596000054
:011597000053
:011598000052
:011599000051
:01159A000050
:01159B00004F
:01159C00004E
:01159D00004D
:01159E00004C
:01159F00004B
:0115A000004A
:0115A1000049
:0115A2000048
:0115A3000047
:0115A4000046
:0115A5000045
:0115A6000044
:0115A7000043
:0115A8000042
:0115A9000041
:0115AA000040
:0115AB00003F
:0115AC00003E
:0115AD00003D
:0115AE00003C
:0115AF00003B
:0115B000003A
:0115B1000039
:0115B2000038
:0115B3000037
:0115B4000036
:0115B5000035
:0115B6000034
:0115B7000033
:0115B8000032
:0115B9000031
:0115BA000030
:0115BB00002F
:0115BC00002E
:0115BD00002D
:0115BE00002C
:0115BF00002B
:0115C000002A
:0115C1000029
:0115C2000028
:0115C3000027
:0115C4000026
:0115C5000025
:0115C6000024
:0115C7000023
:0115C8000022
:0115C9000021
:0115CA000020
:0115CB00001F
:0115CC00001E
:0115CD00001D
:0115CE00001C
:0115CF00001B
:0115D000001A
:0115D1000019
:0115D2000018
:0115D3000017
:0115D4000016
:0115D5000015
:0115D6000014
:0115D7000013
:0115D8000012
:0115D9000011
:0115DA000010
:0115DB00000F
:0115DC00000E
:0115DD00000D
:0115DE00000C
:0115DF00000B
:0115E000000A
:0115E1000009
:0115E2000008
:0115E3000007
:0115E4000006
:0115E5000005
:0115E6000004
:0115E7000003
:0115E8000002
:0115E9000001
:0115EA000000
:0115EB0000FF
:0115EC0000FE
:0115ED0000FD
:0115EE0000FC
:0115EF0000FB
:0115F00000FA
:0115F10000F9
:0115F20000F8
:0115F30000F7
:0115F40000F6
:0115F50000F5
:0115F60000F4
:0115F70000F3
:0115F80000F2
:0115F90000F1
:0115FA0000F0
:0115FB0000EF
:0115FC0000EE
:0115FD0000ED
:0115FE0000EC
:0115FF0000EB
:0116000000E9
:0116010000E8
:0116020000E7
:0116030000E6
:0116040000E5
:0116050000E4
:0116060000E3
:0116070000E2
:0116080000E1
:0116090000E0
:01160A0000DF
:01160B0000DE
:01160C0000DD
:01160D0000DC
:01160E0000DB
:01160F0000DA
:0116100000D9
:0116110000D8
:0116120000D7
:0116130000D6
:0116140000D5
:0116150000D4
:0116160000D3
:0116170000D2
:0116180000D1
:0116190000D0
:01161A0000CF
:01161B0000CE
:01161C0000CD
:01161D0000CC
:01161E0000CB
:01161F0000CA
:0116200000C9
:0116210000C8
:0116220000C7
:0116230000C6
:0116240000C5
:0116250000C4
:0116260000C3
:0116270000C2
:0116280000C1
:0116290000C0
:01162A0000BF
:01162B0000BE
:01162C0000BD
:01162D0000BC
:01162E0000BB
:01162F0000BA
:0116300000B9
:0116310000B8
:0116320000B7
:0116330000B6
:0116340000B5
:0116350000B4
:0116360000B3
:0116370000B2
:0116380000B1
:0116390000B0
:01163A0000AF
:01163B0000AE
:01163C0000AD
:01163D0000AC
:01163E0000AB
:01163F0000AA
:0116400000A9
:0116410000A8
:0116420000A7
:0116430000A6
:0116440000A5
:0116450000A4
:0116460000A3
:0116470000A2
:0116480000A1
:0116490000A0
:01164A00009F
:01164B00009E
:01164C00009D
:01164D00009C
:01164E00009B
:01164F00009A
:011650000099
:011651000098
:011652000097
:011653000096
:011654000095
:011655000094
:011656000093
:011657000092
:011658000091
:011659000090
:01165A00008F
:01165B00008E
:01165C00008D
:01165D00008C
:01165E00008B
:01165F00008A
:011660000089
:011661000088
:011662000087
:011663000086
:011664000085
:011665000084
:011666000083
:011667000082
:011668000081
:011669000080
:01166A00007F
:01166B00007E
:01166C00007D
:01166D00007C
:01166E00007B
:01166F00007A
:011670000079
:011671000078
:011672000077
:011673000076
:011674000075
:011675000074
:011676000073
:011677000072
:011678000071
:011679000070
:01167A00006F
:01167B00006E
:01167C00006D
:01167D00006C
:01167E00006B
:01167F00006A
:011680000069
:011681000068
:011682000067
:011683000066
:011684000065
:011685000064
:011686000063
:011687000062
:011688000061
:011689000060
:01168A00005F
:01168B00005E
:01168C00005D
:01168D00005C
:01168E00005B
:01168F00005A
:011690000059
:011691000058
:011692000057
:011693000056
:011694000055
:011695000054
:011696000053
:011697000052
:011698000051
:011699000050
:01169A00004F
:01169B00004E
:01169C00004D
:01169D00004C
:01169E00004B
:01169F00004A
:0116A0000049
:0116A1000048
:0116A2000047
:0116A3000046
:0116A4000045
:0116A5000044
:0116A6000043
:0116A7000042
:0116A8000041
:0116A9000040
:0116AA00003F
:0116AB00003E
:0116AC00003D
:0116AD00003C
:0116AE00003B
:0116AF00003A
:0116B0000039
:0116B1000038
:0116B2000037
:0116B3000036
:0116B4000035
:0116B5000034
:0116B6000033
:0116B7000032
:0116B8000031
:0116B9000030
:0116BA00002F
:0116BB00002E
:0116BC00002D
:0116BD00002C
:0116BE00002B
:0116BF00002A
:0116C0000029
:0116C1000028
:0116C2000027
:0116C3000026
:0116C4000025
:0116C5000024
:0116C6000023
:0116C7000022
:0116C8000021
:0116C9000020
:0116CA00001F
:0116CB00001E
:0116CC00001D
:0116CD00001C
:0116CE00001B
:0116CF00001A
:0116D0000019
:0116D1000018
:0116D2000017
:0116D3000016
:0116D4000015
:0116D5000014
:0116D6000013
:0116D7000012
:0116D8000011
:0116D9000010
:0116DA00000F
:0116DB00000E
:0116DC00000D
:0116DD00000C
:0116DE00000B
:0116DF00000A
:0116E0000009
:0116E1000008
:0116E2000007
:0116E3000006
:0116E4000005
:0116E5000004
:0116E6000003
:0116E7000002
:0116E8000001
:0116E9000000
:0116EA0000FF
:0116EB0000FE
:0116EC0000FD
:0116ED0000FC
:0116EE0000FB
:0116EF0000FA
:0116F00000F9
:0116F10000F8
:0116F20000F7
:0116F30000F6
:0116F40000F5
:0116F50000F4
:0116F60000F3
:0116F70000F2
:0116F80000F1
:0116F90000F0
:0116FA0000EF
:0116FB0000EE
:0116FC0000ED
:0116FD0000EC
:0116FE0000EB
:0116FF0000EA
:0117000000E8
:0117010000E7
:0117020000E6
:0117030000E5
:0117040000E4
:0117050000E3
:0117060000E2
:0117070000E1
:0117080000E0
:0117090000DF
:01170A0000DE
:01170B0000DD
:01170C0000DC
:01170D0000DB
:01170E0000DA
:01170F0000D9
:0117100000D8
:0117110000D7
:0117120000D6
:0117130000D5
:0117140000D4
:0117150000D3
:0117160000D2
:0117170000D1
:0117180000D0
:0117190000CF
:01171A0000CE
:01171B0000CD
:01171C0000CC
:01171D0000CB
:01171E0000CA
:01171F0000C9
:0117200000C8
:0117210000C7
:0117220000C6
:0117230000C5
:0117240000C4
:0117250000C3
:0117260000C2
:0117270000C1
:0117280000C0
:0117290000BF
:01172A0000BE
:01172B0000BD
:01172C0000BC
:01172D0000BB
:01172E0000BA
:01172F0000B9
:0117300000B8
:0117310000B7
:0117320000B6
:0117330000B5
:0117340000B4
:0117350000B3
:0117360000B2
:0117370000B1
:0117380000B0
:0117390000AF
:01173A0000AE
:01173B0000AD
:01173C0000AC
:01173D0000AB
:01173E0000AA
:01173F0000A9
:0117400000A8
:0117410000A7
:0117420000A6
:0117430000A5
:0117440000A4
:0117450000A3
:0117460000A2
:0117470000A1
:0117480000A0
:01174900009F
:01174A00009E
:01174B00009D
:01174C00009C
:01174D00009B
:01174E00009A
:01174F000099
:011750000098
:011751000097
:011752000096
:011753000095
:011754000094
:011755000093
:011756000092
:011757000091
:011758000090
:01175900008F
:01175A00008E
:01175B00008D
:01175C00008C
:01175D00008B
:01175E00008A
:01175F000089
:011760000088
:011761000087
:011762000086
:011763000085
:011764000084
:011765000083
:011766000082
:011767000081
:011768000080
:01176900007F
:01176A00007E
:01176B00007D
:01176C00007C
:01176D00007B
:01176E00007A
:01176F000079
:011770000078
:011771000077
:011772000076
:011773000075
:011774000074
:011775000073
:011776000072
:011777000071
:011778000070
:01177900006F
:01177A00006E
:01177B00006D
:01177C00006C
:01177D00006B
:01177E00006A
:01177F000069
:011780000068
:011781000067
:011782000066
:011783000065
:011784000064
:011785000063
:011786000062
:011787000061
:011788000060
:01178900005F
:01178A00005E
:01178B00005D
:01178C00005C
:01178D00005B
:01178E00005A
:01178F000059
:011790000058
:011791000057
:011792000056
:011793000055
:011794000054
:011795000053
:011796000052
:011797000051
:011798000050
:01179900004F
:01179A00004E
:01179B00004D
:01179C00004C
:01179D00004B
:01179E00004A
:01179F000049
:0117A0000048
:0117A1000047
:0117A2000046
:0117A3000045
:0117A4000044
:0117A5000043
:0117A6000042
:0117A7000041
:0117A8000040
:0117A900003F
:0117AA00003E
:0117AB00003D
:0117AC00003C
:0117AD00003B
:0117AE00003A
:0117AF000039
:0117B0000038
:0117B1000037
:0117B2000036
:0117B3000035
:0117B4000034
:0117B5000033
:0117B6000032
:0117B7000031
:0117B8000030
:0117B900002F
:0117BA00002E
:0117BB00002D
:0117BC00002C
:0117BD00002B
:0117BE00002A
:0117BF000029
:0117C0000028
:0117C1000027
:0117C2000026
:0117C3000025
:0117C4000024
:0117C5000023
:0117C6000022
:0117C7000021
:0117C8000020
:0117C900001F
:0117CA00001E
:0117CB00001D
:0117CC00001C
:0117CD00001B
:0117CE00001A
:0117CF000019
:0117D0000018
:0117D1000017
:0117D2000016
:0117D3000015
:0117D4000014
:0117D5000013
:0117D6000012
:0117D7000011
:0117D8000010
:0117D900000F
:0117DA00000E
:0117DB00000D
:0117DC00000C
:0117DD00000B
:0117DE00000A
:0117DF000009
:0117E0000008
:0117E1000007
:0117E2000006
:0117E3000005
:0117E4000004
:0117E5000003
:0117E6000002
:0117E7000001
:0117E8000000
:0117E90000FF
:0117EA0000FE
:0117EB0000FD
:0117EC0000FC
:0117ED0000FB
:0117EE0000FA
:0117EF0000F9
:0117F00000F8
:0117F10000F7
:0117F20000F6
:0117F30000F5
:0117F40000F4
:0117F50000F3
:0117F60000F2
:0117F70000F1
:0117F80000F0
:0117F90000EF
:0117FA0000EE
:0117FB0000ED
:0117FC0000EC
:0117FD0000EB
:0117FE0000EA
:0117FF0000E9
:0118000000E7
:0118010000E6
:0118020000E5
:0118030000E4
:0118040000E3
:0118050000E2
:0118060000E1
:0118070000E0
:0118080000DF
:0118090000DE
:01180A0000DD
:01180B0000DC
:01180C0000DB
:01180D0000DA
:01180E0000D9
:01180F0000D8
:0118100000D7
:0118110000D6
:0118120000D5
:0118130000D4
:0118140000D3
:0118150000D2
:0118160000D1
:0118170000D0
:0118180000CF
:0118190000CE
:01181A0000CD
:01181B0000CC
:01181C0000CB
:01181D0000CA
:01181E0000C9
:01181F0000C8
:0118200000C7
:0118210000C6
:0118220000C5
:0118230000C4
:0118240000C3
:0118250000C2
:0118260000C1
:0118270000C0
:0118280000BF
:0118290000BE
:01182A0000BD
:01182B0000BC
:01182C0000BB
:01182D0000BA
:01182E0000B9
:01182F0000B8
:0118300000B7
:0118310000B6
:0118320000B5
:0118330000B4
:0118340000B3
:0118350000B2
:0118360000B1
:0118370000B0
:0118380000AF
:0118390000AE
:01183A0000AD
:01183B0000AC
:01183C0000AB
:01183D0000AA
:01183E0000A9
:01183F0000A8
:0118400000A7
:0118410000A6
:0118420000A5
:0118430000A4
:0118440000A3
:0118450000A2
:0118460000A1
:0118470000A0
:01184800009F
:01184900009E
:01184A00009D
:01184B00009C
:01184C00009B
:01184D00009A
:01184E000099
:01184F000098
:011850000097
:011851000096
:011852000095
:011853000094
:011854000093
:011855000092
:011856000091
:011857000090
:01185800008F
:01185900008E
:01185A00008D
:01185B00008C
:01185C00008B
:01185D00008A
:01185E000089
:01185F000088
:011860000087
:011861000086
:011862000085
:011863000084
:011864000083
:011865000082
:011866000081
:011867000080
:01186800007F
:01186900007E
:01186A00007D
:01186B00007C
:01186C00007B
:01186D00007A
:01186E000079
:01186F000078
:011870000077
:011871000076
:011872000075
:011873000074
:011874000073
:011875000072
:011876000071
:011877000070
:01187800006F
:01187900006E
:01187A00006D
:01187B00006C
:01187C00006B
:01187D00006A
:01187E000069
:01187F000068
:011880000067
:011881000066
:011882000065
:011883000064
:011884000063
:011885000062
:011886000061
:011887000060
:01188800005F
:01188900005E
:01188A00005D
:01188B00005C
:01188C00005B
:01188D00005A
:01188E000059
:01188F000058
:011890000057
:011891000056
:011892000055
:011893000054
:011894000053
:011895000052
:011896000051
:011897000050
:01189800004F
:01189900004E
:01189A00004D
:01189B00004C
:01189C00004B
:01189D00004A
:01189E000049
:01189F000048
:0118A0000047
:0118A1000046
:0118A2000045
:0118A3000044
:0118A4000043
:0118A5000042
:0118A6000041
:0118A7000040
:0118A800003F
:0118A900003E
:0118AA00003D
:0118AB00003C
:0118AC00003B
:0118AD00003A
:0118AE000039
:0118AF000038
:0118B0000037
:0118B1000036
:0118B2000035
:0118B3000034
:0118B4000033
:0118B5000032
:0118B6000031
:0118B7000030
:0118B800002F
:0118B900002E
:0118BA00002D
:0118BB00002C
:0118BC00002B
:0118BD00002A
:0118BE000029
:0118BF000028
:0118C0000027
:0118C1000026
:0118C2000025
:0118C3000024
:0118C4000023
:0118C5000022
:0118C6000021
:0118C7000020
:0118C800001F
:0118C900001E
:0118CA00001D
:0118CB00001C
:0118CC00001B
:0118CD00001A
:0118CE000019
:0118CF000018
:0118D0000017
:0118D1000016
:0118D2000015
:0118D3000014
:0118D4000013
:0118D5000012
:0118D6000011
:0118D7000010
:0118D800000F
:0118D900000E
:0118DA00000D
:0118DB00000C
:0118DC00000B
:0118DD00000A
:0118DE000009
:0118DF000008
:0118E0000007
:0118E1000006
:0118E2000005
:0118E3000004
:0118E4000003
:0118E5000002
:0118E6000001
:0118E7000000
:0118E80000FF
:0118E90000FE
:0118EA0000FD
:0118EB0000FC
:0118EC0000FB
:0118ED0000FA
:0118EE0000F9
:0118EF0000F8
:0118F00000F7
:0118F10000F6
:0118F20000F5
:0118F30000F4
:0118F40000F3
:0118F50000F2
:0118F60000F1
:0118F70000F0
:0118F80000EF
:0118F90000EE
:0118FA0000ED
:0118FB0000EC
:0118FC0000EB
:0118FD0000EA
:0118FE0000E9
:0118FF0000E8
:0119000000E6
:0119010000E5
:0119020000E4
:0119030000E3
:0119040000E2
:0119050000E1
:0119060000E0
:0119070000DF
:0119080000DE
:0119090000DD
:01190A0000DC
:01190B0000DB
:01190C0000DA
:01190D0000D9
:01190E0000D8
:01190F0000D7
:0119100000D6
:0119110000D5
:0119120000D4
:0119130000D3
:0119140000D2
:0119150000D1
:0119160000D0
:0119170000CF
:0119180000CE
:0119190000CD
:01191A0000CC
:01191B0000CB
:01191C0000CA
:01191D0000C9
:01191E0000C8
:01191F0000C7
:0119200000C6
:0119210000C5
:0119220000C4
:0119230000C3
:0119240000C2
:0119250000C1
:0119260000C0
:0119270000BF
:0119280000BE
:0119290000BD
:01192A0000BC
:01192B0000BB
:01192C0000BA
:01192D0000B9
:01192E0000B8
:01192F0000B7
:0119300000B6
:0119310000B5
:0119320000B4
:0119330000B3
:0119340000B2
:0119350000B1
:0119360000B0
:0119370000AF
:0119380000AE
:0119390000AD
:01193A0000AC
:01193B0000AB
:01193C0000AA
:01193D0000A9
:01193E0000A8
:01193F0000A7
:0119400000A6
:0119410000A5
:0119420000A4
:0119430000A3
:0119440000A2
:0119450000A1
:0119460000A0
:01194700009F
:01194800009E
:01194900009D
:01194A00009C
:01194B00009B
:01194C00009A
:01194D000099
:01194E000098
:01194F000097
:011950000096
:011951000095
:011952000094
:011953000093
:011954000092
:011955000091
:011956000090
:01195700008F
:01195800008E
:01195900008D
:01195A00008C
:01195B00008B
:01195C00008A
:01195D000089
:01195E000088
:01195F000087
:011960000086
:011961000085
:011962000084
:011963000083
:011964000082
:011965000081
:011966000080
:01196700007F
:01196800007E
:01196900007D
:01196A00007C
:01196B00007B
:01196C00007A
:01196D000079
:01196E000078
:01196F000077
:011970000076
:011971000075
:011972000074
:011973000073
:011974000072
:011975000071
:011976000070
:01197700006F
:01197800006E
:01197900006D
:01197A00006C
:01197B00006B
:01197C00006A
:01197D000069
:01197E000068
:01197F000067
:011980000066
:011981000065
:011982000064
:011983000063
:011984000062
:011985000061
:011986000060
:01198700005F
:01198800005E
:01198900005D
:01198A00005C
:01198B00005B
:01198C00005A
:01198D000059
:01198E000058
:01198F000057
:011990000056
:011991000055
:011992000054
:011993000053
:011994000052
:011995000051
:011996000050
:01199700004F
:01199800004E
:01199900004D
:01199A00004C
:01199B00004B
:01199C00004A
:01199D000049
:01199E000048
:01199F000047
:0119A0000046
:0119A1000045
:0119A2000044
:0119A3000043
:0119A4000042
:0119A5000041
:0119A6000040
:0119A700003F
:0119A800003E
:0119A900003D
:0119AA00003C
:0119AB00003B
:0119AC00003A
:0119AD000039
:0119AE000038
:0119AF000037
:0119B0000036
:0119B1000035
:0119B2000034
:0119B3000033
:0119B4000032
:0119B5000031
:0119B6000030
:0119B700002F
:0119B800002E
:0119B900002D
:0119BA00002C
:0119BB00002B
:0119BC00002A
:0119BD000029
:0119BE000028
:0119BF000027
:0119C0000026
:0119C1000025
:0119C2000024
:0119C3000023
:0119C4000022
:0119C5000021
:0119C6000020
:0119C700001F
:0119C800001E
:0119C900001D
:0119CA00001C
:0119CB00001B
:0119CC00001A
:0119CD000019
:0119CE000018
:0119CF000017
:0119D0000016
:0119D1000015
:0119D2000014
:0119D3000013
:0119D4000012
:0119D5000011
:0119D6000010
:0119D700000F
:0119D800000E
:0119D900000D
:0119DA00000C
:0119DB00000B
:0119DC00000A
:0119DD000009
:0119DE000008
:0119DF000007
:0119E0000006
:0119E1000005
:0119E2000004
:0119E3000003
:0119E4000002
:0119E5000001
:0119E6000000
:0119E70000FF
:0119E80000FE
:0119E90000FD
:0119EA0000FC
:0119EB0000FB
:0119EC0000FA
:0119ED0000F9
:0119EE0000F8
:0119EF0000F7
:0119F00000F6
:0119F10000F5
:0119F20000F4
:0119F30000F3
:0119F40000F2
:0119F50000F1
:0119F60000F0
:0119F70000EF
:0119F80000EE
:0119F90000ED
:0119FA0000EC
:0119FB0000EB
:0119FC0000EA
:0119FD0000E9
:0119FE0000E8
:0119FF0000E7
:011A000000E5
:011A010000E4
:011A020000E3
:011A030000E2
:011A040000E1
:011A050000E0
:011A060000DF
:011A070000DE
:011A080000DD
:011A090000DC
:011A0A0000DB
:011A0B0000DA
:011A0C0000D9
:011A0D0000D8
:011A0E0000D7
:011A0F0000D6
:011A100000D5
:011A110000D4
:011A120000D3
:011A130000D2
:011A140000D1
:011A150000D0
:011A160000CF
:011A170000CE
:011A180000CD
:011A190000CC
:011A1A0000CB
:011A1B0000CA
:011A1C0000C9
:011A1D0000C8
:011A1E0000C7
:011A1F0000C6
:011A200000C5
:011A210000C4
:011A220000C3
:011A230000C2
:011A240000C1
:011A250000C0
:011A260000BF
:011A270000BE
:011A280000BD
:011A290000BC
:011A2A0000BB
:011A2B0000BA
:011A2C0000B9
:011A2D0000B8
:011A2E0000B7
:011A2F0000B6
:011A300000B5
:011A310000B4
:011A320000B3
:011A330000B2
:011A340000B1
:011A350000B0
:011A360000AF
:011A370000AE
:011A380000AD
:011A390000AC
:011A3A0000AB
:011A3B0000AA
:011A3C0000A9
:011A3D0000A8
:011A3E0000A7
:011A3F0000A6
:011A400000A5
:011A410000A4
:011A420000A3
:011A430000A2
:011A440000A1
:011A450000A0
:011A4600009F
:011A4700009E
:011A4800009D
:011A4900009C
:011A4A00009B
:011A4B00009A
:011A4C000099
:011A4D000098
:011A4E000097
:011A4F000096
:011A50000095
:011A51000094
:011A52000093
:011A53000092
:011A54000091
:011A55000090
:011A5600008F
:011A5700008E
:011A5800008D
:011A5900008C
:011A5A00008B
:011A5B00008A
:011A5C000089
:011A5D000088
:011A5E000087
:011A5F000086
:011A60000085
:011A61000084
:011A62000083
:011A63000082
:011A64000081
:011A65000080
:011A6600007F
:011A6700007E
:011A6800007D
:011A6900007C
:011A6A00007B
:011A6B00007A
:011A6C000079
:011A6D000078
:011A6E000077
:011A6F000076
:011A70000075
:011A71000074
:011A72000073
:011A73000072
:011A74000071
:011A75000070
:011A7600006F
:011A7700006E
:011A7800006D
:011A7900006C
:011A7A00006B
:011A7B00006A
:011A7C000069
:011A7D000068
:011A7E000067
:011A7F000066
:011A80000065
:011A81000064
:011A82000063
:011A83000062
:011A84000061
:011A85000060
:011A8600005F
:011A8700005E
:011A8800005D
:011A8900005C
:011A8A00005B
:011A8B00005A
:011A8C000059
:011A8D000058
:011A8E000057
:011A8F000056
:011A90000055
:011A91000054
:011A92000053
:011A93000052
:011A94000051
:011A95000050
:011A9600004F
:011A9700004E
:011A9800004D
:011A9900004C
:011A9A00004B
:011A9B00004A
:011A9C000049
:011A9D000048
:011A9E000047
:011A9F000046
:011AA0000045
:011AA1000044
:011AA2000043
:011AA3000042
:011AA4000041
:011AA5000040
:011AA600003F
:011AA700003E
:011AA800003D
:011AA900003C
:011AAA00003B
:011AAB00003A
:011AAC000039
:011AAD000038
:011AAE000037
:011AAF000036
:011AB0000035
:011AB1000034
:011AB2000033
:011AB3000032
:011AB4000031
:011AB5000030
:011AB600002F
:011AB700002E
:011AB800002D
:011AB900002C
:011ABA00002B
:011ABB00002A
:011ABC000029
:011ABD000028
:011ABE000027
:011ABF000026
:011AC0000025
:011AC1000024
:011AC2000023
:011AC3000022
:011AC4000021
:011AC5000020
:011AC600001F
:011AC700001E
:011AC800001D
:011AC900001C
:011ACA00001B
:011ACB00001A
:011ACC000019
:011ACD000018
:011ACE000017
:011ACF000016
:011AD0000015
:011AD1000014
:011AD2000013
:011AD3000012
:011AD4000011
:011AD5000010
:011AD600000F
:011AD700000E
:011AD800000D
:011AD900000C
:011ADA00000B
:011ADB00000A
:011ADC000009
:011ADD000008
:011ADE000007
:011ADF000006
:011AE0000005
:011AE1000004
:011AE2000003
:011AE3000002
:011AE4000001
:011AE5000000
:011AE60000FF
:011AE70000FE
:011AE80000FD
:011AE90000FC
:011AEA0000FB
:011AEB0000FA
:011AEC0000F9
:011AED0000F8
:011AEE0000F7
:011AEF0000F6
:011AF00000F5
:011AF10000F4
:011AF20000F3
:011AF30000F2
:011AF40000F1
:011AF50000F0
:011AF60000EF
:011AF70000EE
:011AF80000ED
:011AF90000EC
:011AFA0000EB
:011AFB0000EA
:011AFC0000E9
:011AFD0000E8
:011AFE0000E7
:011AFF0000E6
:011B000000E4
:011B010000E3
:011B020000E2
:011B030000E1
:011B040000E0
:011B050000DF
:011B060000DE
:011B070000DD
:011B080000DC
:011B090000DB
:011B0A0000DA
:011B0B0000D9
:011B0C0000D8
:011B0D0000D7
:011B0E0000D6
:011B0F0000D5
:011B100000D4
:011B110000D3
:011B120000D2
:011B130000D1
:011B140000D0
:011B150000CF
:011B160000CE
:011B170000CD
:011B180000CC
:011B190000CB
:011B1A0000CA
:011B1B0000C9
:011B1C0000C8
:011B1D0000C7
:011B1E0000C6
:011B1F0000C5
:011B200000C4
:011B210000C3
:011B220000C2
:011B230000C1
:011B240000C0
:011B250000BF
:011B260000BE
:011B270000BD
:011B280000BC
:011B290000BB
:011B2A0000BA
:011B2B0000B9
:011B2C0000B8
:011B2D0000B7
:011B2E0000B6
:011B2F0000B5
:011B300000B4
:011B310000B3
:011B320000B2
:011B330000B1
:011B340000B0
:011B350000AF
:011B360000AE
:011B370000AD
:011B380000AC
:011B390000AB
:011B3A0000AA
:011B3B0000A9
:011B3C0000A8
:011B3D0000A7
:011B3E0000A6
:011B3F0000A5
:011B400000A4
:011B410000A3
:011B420000A2
:011B430000A1
:011B440000A0
:011B4500009F
:011B4600009E
:011B4700009D
:011B4800009C
:011B4900009B
:011B4A00009A
:011B4B000099
:011B4C000098
:011B4D000097
:011B4E000096
:011B4F000095
:011B50000094
:011B51000093
:011B52000092
:011B53000091
:011B54000090
:011B5500008F
:011B5600008E
:011B5700008D
:011B5800008C
:011B5900008B
:011B5A00008A
:011B5B000089
:011B5C000088
:011B5D000087
:011B5E000086
:011B5F000085
:011B60000084
:011B61000083
:011B62000082
:011B63000081
:011B64000080
:011B6500007F
:011B6600007E
:011B6700007D
:011B6800007C
:011B6900007B
:011B6A00007A
:011B6B000079
:011B6C000078
:011B6D000077
:011B6E000076
:011B6F000075
:011B70000074
:011B71000073
:011B72000072
:011B73000071
:011B74000070
:011B7500006F
:011B7600006E
:011B7700006D
:011B7800006C
:011B7900006B
:011B7A00006A
:011B7B000069
:011B7C000068
:011B7D000067
:011B7E000066
:011B7F000065
:011B80000064
:011B81000063
:011B82000062
:011B83000061
:011B84000060
:011B8500005F
:011B8600005E
:011B8700005D
:011B8800005C
:011B8900005B
:011B8A00005A
:011B8B000059
:011B8C000058
:011B8D000057
:011B8E000056
:011B8F000055
:011B90000054
:011B91000053
:011B92000052
:011B93000051
:011B94000050
:011B9500004F
:011B9600004E
:011B9700004D
:011B9800004C
:011B9900004B
:011B9A00004A
:011B9B000049
:011B9C000048
:011B9D000047
:011B9E000046
:011B9F000045
:011BA0000044
:011BA1000043
:011BA2000042
:011BA3000041
:011BA4000040
:011BA500003F
:011BA600003E
:011BA700003D
:011BA800003C
:011BA900003B
:011BAA00003A
:011BAB000039
:011BAC000038
:011BAD000037
:011BAE000036
:011BAF000035
:011BB0000034
:011BB1000033
:011BB2000032
:011BB3000031
:011BB4000030
:011BB500002F
:011BB600002E
:011BB700002D
:011BB800002C
:011BB900002B
:011BBA00002A
:011BBB000029
:011BBC000028
:011BBD000027
:011BBE000026
:011BBF000025
:011BC0000024
:011BC1000023
:011BC2000022
:011BC3000021
:011BC4000020
:011BC500001F
:011BC600001E
:011BC700001D
:011BC800001C
:011BC900001B
:011BCA00001A
:011BCB000019
:011BCC000018
:011BCD000017
:011BCE000016
:011BCF000015
:011BD0000014
:011BD1000013
:011BD2000012
:011BD3000011
:011BD4000010
:011BD500000F
:011BD600000E
:011BD700000D
:011BD800000C
:011BD900000B
:011BDA00000A
:011BDB000009
:011BDC000008
:011BDD000007
:011BDE000006
:011BDF000005
:011BE0000004
:011BE1000003
:011BE2000002
:011BE3000001
:011BE4000000
:011BE50000FF
:011BE60000FE
:011BE70000FD
:011BE80000FC
:011BE90000FB
:011BEA0000FA
:011BEB0000F9
:011BEC0000F8
:011BED0000F7
:011BEE0000F6
:011BEF0000F5
:011BF00000F4
:011BF10000F3
:011BF20000F2
:011BF30000F1
:011BF40000F0
:011BF50000EF
:011BF60000EE
:011BF70000ED
:011BF80000EC
:011BF90000EB
:011BFA0000EA
:011BFB0000E9
:011BFC0000E8
:011BFD0000E7
:011BFE0000E6
:011BFF0000E5
:011C000000E3
:011C010000E2
:011C020000E1
:011C030000E0
:011C040000DF
:011C050000DE
:011C060000DD
:011C070000DC
:011C080000DB
:011C090000DA
:011C0A0000D9
:011C0B0000D8
:011C0C0000D7
:011C0D0000D6
:011C0E0000D5
:011C0F0000D4
:011C100000D3
:011C110000D2
:011C120000D1
:011C130000D0
:011C140000CF
:011C150000CE
:011C160000CD
:011C170000CC
:011C180000CB
:011C190000CA
:011C1A0000C9
:011C1B0000C8
:011C1C0000C7
:011C1D0000C6
:011C1E0000C5
:011C1F0000C4
:011C200000C3
:011C210000C2
:011C220000C1
:011C230000C0
:011C240000BF
:011C250000BE
:011C260000BD
:011C270000BC
:011C280000BB
:011C290000BA
:011C2A0000B9
:011C2B0000B8
:011C2C0000B7
:011C2D0000B6
:011C2E0000B5
:011C2F0000B4
:011C300000B3
:011C310000B2
:011C320000B1
:011C330000B0
:011C340000AF
:011C350000AE
:011C360000AD
:011C370000AC
:011C380000AB
:011C390000AA
:011C3A0000A9
:011C3B0000A8
:011C3C0000A7
:011C3D0000A6
:011C3E0000A5
:011C3F0000A4
:011C400000A3
:011C410000A2
:011C420000A1
:011C430000A0
:011C4400009F
:011C4500009E
:011C4600009D
:011C4700009C
:011C4800009B
:011C4900009A
:011C4A000099
:011C4B000098
:011C4C000097
:011C4D000096
:011C4E000095
:011C4F000094
:011C50000093
:011C51000092
:011C52000091
:011C53000090
:011C5400008F
:011C5500008E
:011C5600008D
:011C5700008C
:011C5800008B
:011C5900008A
:011C5A000089
:011C5B000088
:011C5C000087
:011C5D000086
:011C5E000085
:011C5F000084
:011C60000083
:011C61000082
:011C62000081
:011C63000080
:011C6400007F
:011C6500007E
:011C6600007D
:011C6700007C
:011C6800007B
:011C6900007A
:011C6A000079
:011C6B000078
:011C6C000077
:011C6D000076
:011C6E000075
:011C6F000074
:011C70000073
:011C71000072
:011C72000071
:011C73000070
:011C7400006F
:011C7500006E
:011C7600006D
:011C7700006C
:011C7800006B
:011C7900006A
:011C7A000069
:011C7B000068
:011C7C000067
:011C7D000066
:011C7E000065
:011C7F000064
:011C80000063
:011C81000062
:011C82000061
:011C83000060
:011C8400005F
:011C8500005E
:011C8600005D
:011C8700005C
:011C8800005B
:011C8900005A
:011C8A000059
:011C8B000058
:011C8C000057
:011C8D000056
:011C8E000055
:011C8F000054
:011C90000053
:011C91000052
:011C92000051
:011C93000050
:011C9400004F
:011C9500004E
:011C9600004D
:011C9700004C
:011C9800004B
:011C9900004A
:011C9A000049
:011C9B000048
:011C9C000047
:011C9D000046
:011C9E000045
:011C9F000044
:011CA0000043
:011CA1000042
:011CA2000041
:011CA3000040
:011CA400003F
:011CA500003E
:011CA600003D
:011CA700003C
:011CA800003B
:011CA900003A
:011CAA000039
:011CAB000038
:011CAC000037
:011CAD000036
:011CAE000035
:011CAF000034
:011CB0000033
:011CB1000032
:011CB2000031
:011CB3000030
:011CB400002F
:011CB500002E
:011CB600002D
:011CB700002C
:011CB800002B
:011CB900002A
:011CBA000029
:011CBB000028
:011CBC000027
:011CBD000026
:011CBE000025
:011CBF000024
:011CC0000023
:011CC1000022
:011CC2000021
:011CC3000020
:011CC400001F
:011CC500001E
:011CC600001D
:011CC700001C
:011CC800001B
:011CC900001A
:011CCA000019
:011CCB000018
:011CCC000017
:011CCD000016
:011CCE000015
:011CCF000014
:011CD0000013
:011CD1000012
:011CD2000011
:011CD3000010
:011CD400000F
:011CD500000E
:011CD600000D
:011CD700000C
:011CD800000B
:011CD900000A
:011CDA000009
:011CDB000008
:011CDC000007
:011CDD000006
:011CDE000005
:011CDF000004
:011CE0000003
:011CE1000002
:011CE2000001
:011CE3000000
:011CE40000FF
:011CE50000FE
:011CE60000FD
:011CE70000FC
:011CE80000FB
:011CE90000FA
:011CEA0000F9
:011CEB0000F8
:011CEC0000F7
:011CED0000F6
:011CEE0000F5
:011CEF0000F4
:011CF00000F3
:011CF10000F2
:011CF20000F1
:011CF30000F0
:011CF40000EF
:011CF50000EE
:011CF60000ED
:011CF70000EC
:011CF80000EB
:011CF90000EA
:011CFA0000E9
:011CFB0000E8
:011CFC0000E7
:011CFD0000E6
:011CFE0000E5
:011CFF0000E4
:011D000000E2
:011D010000E1
:011D020000E0
:011D030000DF
:011D040000DE
:011D050000DD
:011D060000DC
:011D070000DB
:011D080000DA
:011D090000D9
:011D0A0000D8
:011D0B0000D7
:011D0C0000D6
:011D0D0000D5
:011D0E0000D4
:011D0F0000D3
:011D100000D2
:011D110000D1
:011D120000D0
:011D130000CF
:011D140000CE
:011D150000CD
:011D160000CC
:011D170000CB
:011D180000CA
:011D190000C9
:011D1A0000C8
:011D1B0000C7
:011D1C0000C6
:011D1D0000C5
:011D1E0000C4
:011D1F0000C3
:011D200000C2
:011D210000C1
:011D220000C0
:011D230000BF
:011D240000BE
:011D250000BD
:011D260000BC
:011D270000BB
:011D280000BA
:011D290000B9
:011D2A0000B8
:011D2B0000B7
:011D2C0000B6
:011D2D0000B5
:011D2E0000B4
:011D2F0000B3
:011D300000B2
:011D310000B1
:011D320000B0
:011D330000AF
:011D340000AE
:011D350000AD
:011D360000AC
:011D370000AB
:011D380000AA
:011D390000A9
:011D3A0000A8
:011D3B0000A7
:011D3C0000A6
:011D3D0000A5
:011D3E0000A4
:011D3F0000A3
:011D400000A2
:011D410000A1
:011D420000A0
:011D4300009F
:011D4400009E
:011D4500009D
:011D4600009C
:011D4700009B
:011D4800009A
:011D49000099
:011D4A000098
:011D4B000097
:011D4C000096
:011D4D000095
:011D4E000094
:011D4F000093
:011D50000092
:011D51000091
:011D52000090
:011D5300008F
:011D5400008E
:011D5500008D
:011D5600008C
:011D5700008B
:011D5800008A
:011D59000089
:011D5A000088
:011D5B000087
:011D5C000086
:011D5D000085
:011D5E000084
:011D5F000083
:011D60000082
:011D61000081
:011D62000080
:011D6300007F
:011D6400007E
:011D6500007D
:011D6600007C
:011D6700007B
:011D6800007A
:011D69000079
:011D6A000078
:011D6B000077
:011D6C000076
:011D6D000075
:011D6E000074
:011D6F000073
:011D70000072
:011D71000071
:011D72000070
:011D7300006F
:011D7400006E
:011D7500006D
:011D7600006C
:011D7700006B
:011D7800006A
:011D79000069
:011D7A000068
:011D7B000067
:011D7C000066
:011D7D000065
:011D7E000064
:011D7F000063
:011D80000062
:011D81000061
:011D82000060
:011D8300005F
:011D8400005E
:011D8500005D
:011D8600005C
:011D8700005B
:011D8800005A
:011D89000059
:011D8A000058
:011D8B000057
:011D8C000056
:011D8D000055
:011D8E000054
:011D8F000053
:011D90000052
:011D91000051
:011D92000050
:011D9300004F
:011D9400004E
:011D9500004D
:011D9600004C
:011D9700004B
:011D9800004A
:011D99000049
:011D9A000048
:011D9B000047
:011D9C000046
:011D9D000045
:011D9E000044
:011D9F000043
:011DA0000042
:011DA1000041
:011DA2000040
:011DA300003F
:011DA400003E
:011DA500003D
:011DA600003C
:011DA700003B
:011DA800003A
:011DA9000039
:011DAA000038
:011DAB000037
:011DAC000036
:011DAD000035
:011DAE000034
:011DAF000033
:011DB0000032
:011DB1000031
:011DB2000030
:011DB300002F
:011DB400002E
:011DB500002D
:011DB600002C
:011DB700002B
:011DB800002A
:011DB9000029
:011DBA000028
:011DBB000027
:011DBC000026
:011DBD000025
:011DBE000024
:011DBF000023
:011DC0000022
:011DC1000021
:011DC2000020
:011DC300001F
:011DC400001E
:011DC500001D
:011DC600001C
:011DC700001B
:011DC800001A
:011DC9000019
:011DCA000018
:011DCB000017
:011DCC000016
:011DCD000015
:011DCE000014
:011DCF000013
:011DD0000012
:011DD1000011
:011DD2000010
:011DD300000F
:011DD400000E
:011DD500000D
:011DD600000C
:011DD700000B
:011DD800000A
:011DD9000009
:011DDA000008
:011DDB000007
:011DDC000006
:011DDD000005
:011DDE000004
:011DDF000003
:011DE0000002
:011DE1000001
:011DE2000000
:011DE30000FF
:011DE40000FE
:011DE50000FD
:011DE60000FC
:011DE70000FB
:011DE80000FA
:011DE90000F9
:011DEA0000F8
:011DEB0000F7
:011DEC0000F6
:011DED0000F5
:011DEE0000F4
:011DEF0000F3
:011DF00000F2
:011DF10000F1
:011DF20000F0
:011DF30000EF
:011DF40000EE
:011DF50000ED
:011DF60000EC
:011DF70000EB
:011DF80000EA
:011DF90000E9
:011DFA0000E8
:011DFB0000E7
:011DFC0000E6
:011DFD0000E5
:011DFE0000E4
:011DFF0000E3
:011E000000E1
:011E010000E0
:011E020000DF
:011E030000DE
:011E040000DD
:011E050000DC
:011E060000DB
:011E070000DA
:011E080000D9
:011E090000D8
:011E0A0000D7
:011E0B0000D6
:011E0C0000D5
:011E0D0000D4
:011E0E0000D3
:011E0F0000D2
:011E100000D1
:011E110000D0
:011E120000CF
:011E130000CE
:011E140000CD
:011E150000CC
:011E160000CB
:011E170000CA
:011E180000C9
:011E190000C8
:011E1A0000C7
:011E1B0000C6
:011E1C0000C5
:011E1D0000C4
:011E1E0000C3
:011E1F0000C2
:011E200000C1
:011E210000C0
:011E220000BF
:011E230000BE
:011E240000BD
:011E250000BC
:011E260000BB
:011E270000BA
:011E280000B9
:011E290000B8
:011E2A0000B7
:011E2B0000B6
:011E2C0000B5
:011E2D0000B4
:011E2E0000B3
:011E2F0000B2
:011E300000B1
:011E310000B0
:011E320000AF
:011E330000AE
:011E340000AD
:011E350000AC
:011E360000AB
:011E370000AA
:011E380000A9
:011E390000A8
:011E3A0000A7
:011E3B0000A6
:011E3C0000A5
:011E3D0000A4
:011E3E0000A3
:011E3F0000A2
:011E400000A1
:011E410000A0
:011E4200009F
:011E4300009E
:011E4400009D
:011E4500009C
:011E4600009B
:011E4700009A
:011E48000099
:011E49000098
:011E4A000097
:011E4B000096
:011E4C000095
:011E4D000094
:011E4E000093
:011E4F000092
:011E50000091
:011E51000090
:011E5200008F
:011E5300008E
:011E5400008D
:011E5500008C
:011E5600008B
:011E5700008A
:011E58000089
:011E59000088
:011E5A000087
:011E5B000086
:011E5C000085
:011E5D000084
:011E5E000083
:011E5F000082
:011E60000081
:011E61000080
:011E6200007F
:011E6300007E
:011E6400007D
:011E6500007C
:011E6600007B
:011E6700007A
:011E68000079
:011E69000078
:011E6A000077
:011E6B000076
:011E6C000075
:011E6D000074
:011E6E000073
:011E6F000072
:011E70000071
:011E71000070
:011E7200006F
:011E7300006E
:011E7400006D
:011E7500006C
:011E7600006B
:011E7700006A
:011E78000069
:011E79000068
:011E7A000067
:011E7B000066
:011E7C000065
:011E7D000064
:011E7E000063
:011E7F000062
:011E80000061
:011E81000060
:011E8200005F
:011E8300005E
:011E8400005D
:011E8500005C
:011E8600005B
:011E8700005A
:011E88000059
:011E89000058
:011E8A000057
:011E8B000056
:011E8C000055
:011E8D000054
:011E8E000053
:011E8F000052
:011E90000051
:011E91000050
:011E9200004F
:011E9300004E
:011E9400004D
:011E9500004C
:011E9600004B
:011E9700004A
:011E98000049
:011E99000048
:011E9A000047
:011E9B000046
:011E9C000045
:011E9D000044
:011E9E000043
:011E9F000042
:011EA0000041
:011EA1000040
:011EA200003F
:011EA300003E
:011EA400003D
:011EA500003C
:011EA600003B
:011EA700003A
:011EA8000039
:011EA9000038
:011EAA000037
:011EAB000036
:011EAC000035
:011EAD000034
:011EAE000033
:011EAF000032
:011EB0000031
:011EB1000030
:011EB200002F
:011EB300002E
:011EB400002D
:011EB500002C
:011EB600002B
:011EB700002A
:011EB8000029
:011EB9000028
:011EBA000027
:011EBB000026
:011EBC000025
:011EBD000024
:011EBE000023
:011EBF000022
:011EC0000021
:011EC1000020
:011EC200001F
:011EC300001E
:011EC400001D
:011EC500001C
:011EC600001B
:011EC700001A
:011EC8000019
:011EC9000018
:011ECA000017
:011ECB000016
:011ECC000015
:011ECD000014
:011ECE000013
:011ECF000012
:011ED0000011
:011ED1000010
:011ED200000F
:011ED300000E
:011ED400000D
:011ED500000C
:011ED600000B
:011ED700000A
:011ED8000009
:011ED9000008
:011EDA000007
:011EDB000006
:011EDC000005
:011EDD000004
:011EDE000003
:011EDF000002
:011EE0000001
:011EE1000000
:011EE20000FF
:011EE30000FE
:011EE40000FD
:011EE50000FC
:011EE60000FB
:011EE70000FA
:011EE80000F9
:011EE90000F8
:011EEA0000F7
:011EEB0000F6
:011EEC0000F5
:011EED0000F4
:011EEE0000F3
:011EEF0000F2
:011EF00000F1
:011EF10000F0
:011EF20000EF
:011EF30000EE
:011EF40000ED
:011EF50000EC
:011EF60000EB
:011EF70000EA
:011EF80000E9
:011EF90000E8
:011EFA0000E7
:011EFB0000E6
:011EFC0000E5
:011EFD0000E4
:011EFE0000E3
:011EFF0000E2
:011F000000E0
:011F010000DF
:011F020000DE
:011F030000DD
:011F040000DC
:011F050000DB
:011F060000DA
:011F070000D9
:011F080000D8
:011F090000D7
:011F0A0000D6
:011F0B0000D5
:011F0C0000D4
:011F0D0000D3
:011F0E0000D2
:011F0F0000D1
:011F100000D0
:011F110000CF
:011F120000CE
:011F130000CD
:011F140000CC
:011F150000CB
:011F160000CA
:011F170000C9
:011F180000C8
:011F190000C7
:011F1A0000C6
:011F1B0000C5
:011F1C0000C4
:011F1D0000C3
:011F1E0000C2
:011F1F0000C1
:011F200000C0
:011F210000BF
:011F220000BE
:011F230000BD
:011F240000BC
:011F250000BB
:011F260000BA
:011F270000B9
:011F280000B8
:011F290000B7
:011F2A0000B6
:011F2B0000B5
:011F2C0000B4
:011F2D0000B3
:011F2E0000B2
:011F2F0000B1
:011F300000B0
:011F310000AF
:011F320000AE
:011F330000AD
:011F340000AC
:011F350000AB
:011F360000AA
:011F370000A9
:011F380000A8
:011F390000A7
:011F3A0000A6
:011F3B0000A5
:011F3C0000A4
:011F3D0000A3
:011F3E0000A2
:011F3F0000A1
:011F400000A0
:011F4100009F
:011F4200009E
:011F4300009D
:011F4400009C
:011F4500009B
:011F4600009A
:011F47000099
:011F48000098
:011F49000097
:011F4A000096
:011F4B000095
:011F4C000094
:011F4D000093
:011F4E000092
:011F4F000091
:011F50000090
:011F5100008F
:011F5200008E
:011F5300008D
:011F5400008C
:011F5500008B
:011F5600008A
:011F57000089
:011F58000088
:011F59000087
:011F5A000086
:011F5B000085
:011F5C000084
:011F5D000083
:011F5E000082
:011F5F000081
:011F60000080
:011F6100007F
:011F6200007E
:011F6300007D
:011F6400007C
:011F6500007B
:011F6600007A
:011F67000079
:011F68000078
:011F69000077
:011F6A000076
:011F6B000075
:011F6C000074
:011F6D000073
:011F6E000072
:011F6F000071
:011F70000070
:011F7100006F
:011F7200006E
:011F7300006D
:011F7400006C
:011F7500006B
:011F7600006A
:011F77000069
:011F78000068
:011F79000067
:011F7A000066
:011F7B000065
:011F7C000064
:011F7D000063
:011F7E000062
:011F7F000061
:011F80000060
:011F8100005F
:011F8200005E
:011F8300005D
:011F8400005C
:011F8500005B
:011F8600005A
:011F87000059
:011F88000058
:011F89000057
:011F8A000056
:011F8B000055
:011F8C000054
:011F8D000053
:011F8E000052
:011F8F000051
:011F90000050
:011F9100004F
:011F9200004E
:011F9300004D
:011F9400004C
:011F9500004B
:011F9600004A
:011F97000049
:011F98000048
:011F99000047
:011F9A000046
:011F9B000045
:011F9C000044
:011F9D000043
:011F9E000042
:011F9F000041
:011FA0000040
:011FA100003F
:011FA200003E
:011FA300003D
:011FA400003C
:011FA500003B
:011FA600003A
:011FA7000039
:011FA8000038
:011FA9000037
:011FAA000036
:011FAB000035
:011FAC000034
:011FAD000033
:011FAE000032
:011FAF000031
:011FB0000030
:011FB100002F
:011FB200002E
:011FB300002D
:011FB400002C
:011FB500002B
:011FB600002A
:011FB7000029
:011FB8000028
:011FB9000027
:011FBA000026
:011FBB000025
:011FBC000024
:011FBD000023
:011FBE000022
:011FBF000021
:011FC0000020
:011FC100001F
:011FC200001E
:011FC300001D
:011FC400001C
:011FC500001B
:011FC600001A
:011FC7000019
:011FC8000018
:011FC9000017
:011FCA000016
:011FCB000015
:011FCC000014
:011FCD000013
:011FCE000012
:011FCF000011
:011FD0000010
:011FD100000F
:011FD200000E
:011FD300000D
:011FD400000C
:011FD500000B
:011FD600000A
:011FD7000009
:011FD8000008
:011FD9000007
:011FDA000006
:011FDB000005
:011FDC000004
:011FDD000003
:011FDE000002
:011FDF000001
:011FE0000000
:011FE10000FF
:011FE20000FE
:011FE30000FD
:011FE40000FC
:011FE50000FB
:011FE60000FA
:011FE70000F9
:011FE80000F8
:011FE90000F7
:011FEA0000F6
:011FEB0000F5
:011FEC0000F4
:011FED0000F3
:011FEE0000F2
:011FEF0000F1
:011FF00000F0
:011FF10000EF
:011FF20000EE
:011FF30000ED
:011FF40000EC
:011FF50000EB
:011FF60000EA
:011FF70000E9
:011FF80000E8
:011FF90000E7
:011FFA0000E6
:011FFB0000E5
:011FFC0000E4
:011FFD0000E3
:011FFE0000E2
:011FFF0000E1
:00000001FF
